:020000040800F2
:100000005806002009740008B1730008B373000893
:10001000B5730008B7730008B9730008000000004A
:10002000000000000000000000000000BB7300089A
:10003000BD73000800000000BF730008C173000812
:1000400075740008797400087D7400087D36000816
:100050008574000889740008AD2E00084930000836
:10006000957400089974000825030008A17400081D
:10007000A5740008A9740008AD740008B1740008E4
:10008000B5740008B9740008BD740008C174000894
:10009000C5740008C9740008CD74000891020008F6
:1000A000D5740008D9740008DD740008DD34000838
:1000B000690B0008E9740008E91A0008F1740008E7
:1000C000F5740008F9740008FD7400080175000853
:1000D00005750008097500080D7500081175000800
:1000E00015750008197500081D75000821750008B0
:1000F0002575000840B24109DFF85C2D012310F09E
:100100001F0013FA00F042F82100704740B2410985
:10011000DFF8482D012310F01F0013FA00F042F819
:100120002100704740B2002809D540B210F00F00FE
:10013000DFF8DC2A8018090100F8041C04E040B252
:10014000DFF81C2D090181547047704700B583B05A
:100150000121012003F0E1FB0121022003F0DDFB7E
:100160000121042003F0D9FB0121082003F0D5FB75
:100170000121102003F0D1FB0121202003F0CDFB51
:100180004FF6FF70009000208DF8060000208DF8DB
:10019000050002208DF8070003208DF8040000A957
:1001A000DFF82C0B03F018FC00A9DFF8280B03F094
:1001B00013FC00A9DFF8200B03F00EFC00A9DFF808
:1001C000440B03F009FC00A9DFF83C0B03F004FC2E
:1001D00048F2FF70009000A9DFF8880C03F0FCFBE8
:1001E00007BD00E0401E0128FCDA704700B583B06F
:1001F0004020009000208DF8060001208DF80500B9
:1002000000208DF8070001208DF8040000A9DFF818
:10021000540C03F0E1FB07BD0068704700B583B0E4
:100220008020009000208DF8040003208DF8050048
:1002300001208DF8070000A9DFF8940A03F0CCFB39
:10024000DFF8480B006850F00100DFF8401B086041
:10025000DFF83C0B006850F48050DFF8341B086076
:10026000DFF8600B006850F08000DFF8581B086072
:10027000DFF8F40B006850F08000DFF8EC1B08603A
:1002800001211720FFF74EFF1720FFF733FF07BDAF
:10029000DFF8640B006850F08000DFF85C1B08603A
:1002A000DFF8C80B0068401CDFF8C01B086070470F
:1002B00000B583B01020009000208DF804000320CA
:1002C0008DF8050001208DF8070000A9DFF8000A6D
:1002D00003F082FBDFF8B40A006850F00100DFF899
:1002E000AC1A0860DFF8A80A006850F00100DFF8D7
:1002F000A01A0860DFF8CC0A006850F01000DFF8A0
:10030000C41A0860DFF8600B006850F01000DFF8D6
:10031000581B086001210A20FFF704FF0A20FFF79D
:10032000E9FE07BDDFF8D00A006850F01000DFF8E2
:10033000C81A0860DFF87C0D0068401CDFF8741DE7
:10034000086070472DE9F04381460E00170098467B
:10035000002400257F1C15E0FFB25FFA89F97820A0
:10036000DFF88C1D00FB091010EB470030F8020C81
:1003700003F0C2FB22002B0003F0CCFB04000D00B5
:10038000761E7F1EF6B2002E02D0FFB2002FE3D100
:10039000B8F1010713E0FFB25FFA89F97820DFF8BE
:1003A000501D00FB091030F8170003F0A5FB2200D8
:1003B0002B0003F0AFFB04000D00761E7F1EF6B28B
:1003C000002EE8D12000290003F018FCBDE8F083DE
:1003D00070B40400002000250FE0D2B2E4B2602522
:1003E000DFF88C6A05FB046515EB820555F8045CA3
:1003F000002D00D42818491E521EC9B2002902D06F
:10040000D2B2002AE9D15A1E0DE0D2B2E4B2602382
:10041000DFF85C5A03FB045353F82250002D00D43C
:100420002818491E521EC9B20029EED170BC70476F
:100430002DE9F04F87B083460020019000208DF811
:1004400000005FF0000A0022002600275FF000088D
:100450005FF000090024002500200021CDE90401FF
:1004600000200021CDE90201DFF8140D00681F28EB
:10047000C0F0AE8000220EE05FFA8BFB6020DFF858
:10048000F01900FB0B1050F8220010F1010F01D001
:100490001AF1010A521C182AEED3DFF8E40C0068A6
:1004A0001E21B0FBF1F00190BAF1000F79D0019854
:1004B000401E8DF800009DF80000824525D21823CB
:1004C000DFF8840B02785146C9B25846C0B2FFF734
:1004D0007FFF03F011FB04000D00504603F00CFBFE
:1004E00002000B002000290003F0B4FB06000F00FF
:1004F0009DF80000B0EB0A0003F0FEFA32003B006A
:1005000003F0E2FCCDE902010DE01823DFF8380B1F
:1005100002789DF800105846C0B2FFF759FF03F06B
:10052000EBFA04000D003C23DFF88C0B0278DFF8B7
:10053000880B0078411CC9B25846C0B2FFF702FFD1
:1005400003F0DAFA804689469DF800003C214843D2
:1005500003F0C8FA02000B002000290003F07AFB28
:1005600006000F00DFF8500B0078D0F13C00401E71
:1005700003F0B8FA32003B0003F0A6FCCDE9040119
:1005800022002B004046494603F0C4FADDE904236B
:1005900003F0C0FADDE9022303F0BCFA06000F0005
:1005A00028E03C23DFF8100B02783C215846C0B20B
:1005B000FFF7C8FE03F0A0FA06000F00019803F051
:1005C0009BFA32003B0003F07FFC06000F0011E0B5
:1005D0003C23DFF8E40A0278DFF8A40B0068C0B21D
:1005E0004100C9B25846C0B2FFF7ACFE03F084FA2E
:1005F00006000F0000205FF0804132003B0003F056
:1006000063FC04000D005FFA8BFBDFF8780B50F8F9
:100610002B0003F067FA22002B0003F055FC0400C6
:100620000D00DFF85C0B0068400003F065FA020083
:100630000B002000290003F00DFB07B0BDE8F08F90
:1006400010B5DFF8700A0068B0F5805F04D3DFF8FA
:10065000640A40F6FF710160DFF810080068B0F529
:10066000805F04D3DFF8040840F6FF710160DFF813
:10067000440A006803F040FADFF8984BD4E90023FD
:1006800003F048FADFF88C2BC2E90001DFF8DC0741
:10069000006803F031FADFF8804BD4E9002303F05F
:1006A00039FADFF8742BC2E90001DFF80C0A007890
:1006B000DFF83C1ADFF8FC29126821F81020DFF877
:1006C000F8090078DFF8281A11EB4000DFF89C17D2
:1006D0000968A0F87810DFF8DC0900210160DFF874
:1006E0008C07002101600020FFF7A2FEDFF82C2B11
:1006F000C2E900010120FFF79BFEDFF8242BC2E9CD
:100700000001DFF81C2BD2E90001DFF8104BD4E91F
:10071000002303F0BBFC14D2DFF8040BD0E9002364
:100720000020DFF8001B03F0CFFBDFF8F04AD4E92C
:10073000002303F08FFA03F061FADFF8EC1A086087
:1007400003E0DFF8E40A63210160DFF8D02AD2E990
:1007500000010022DFF8D43A03F07CFADFF8BC2A6B
:10076000C2E90001DFF8B82AD2E900010022DFF86F
:10077000BC3A03F06FFADFF8A82AC2E90001DFF8FB
:1007800038090078401CDFF830190870DFF82809B4
:1007900000783C282ED13C2300223C210020FFF78A
:1007A000D1FDDFF8A4180978DFF8C42642F821004B
:1007B0003C2300223C210120FFF7C4FDDFF888180C
:1007C0000978DFF8AC2612EB81010866DFF87808BB
:1007D0000078401CDFF870180870DFF86C080078AB
:1007E000182803D1DFF8600800210170DFF8C8087D
:1007F00000210170DFF8640C008840F69F71884288
:1008000006DADFF8580C0088401CDFF8501C08801E
:1008100010BD80B50020DFF8A01801220A70DFF8B3
:10082000D81B3C220A700021080006E0C0B2DFF8A5
:10083000C018002221F81020401CC0B23C28F5DB73
:10084000002008E0C0B2DFF8A81811EB4001002238
:10085000A1F87820401CC0B23C28F3DBDFF8540834
:1008600000210160DFF8040600210160DFF8AC0917
:1008700000220023C0E90023DFF8A409002200239E
:10088000C0E90023002007E0C0B2DFF8E4155FF004
:10089000FF3241F82020401CC0B21828F4DB0020B1
:1008A00008E0C0B2DFF8C81511EB80015FF0FF323D
:1008B0000A66401CC0B21828F3DBDFF88C07002161
:1008C0000170DFF8980B00210180DFF8480CFFF77A
:1008D000A3FCDFF8B0180860DFF83C0CFFF79CFCC5
:1008E000DFF8A0184860DFF8340CFFF795FCDFF85C
:1008F000301C0870DFF82C0CFFF78EFCDFF8201C92
:100900004870DFF8240CFFF787FCDFF8201C087024
:10091000DFF81C0CFFF780FCDFF8101C4870DFF8D4
:10092000140CFFF779FCDFF8241D087001BD80B5B9
:100930000A20FFF7DFFBDFF85804006850F00100E1
:10094000DFF84C1408601720FFF7D4FBDFF84004F1
:10095000006850F48050DFF83814086001BD80B59D
:10096000DFF82C04006840084000DFF82414086019
:100970000A20FFF7CBFBDFF81804006830F4805042
:10098000DFF80C1408601720FFF7C0FB01BD10B59D
:100990000400E4B2002C03D1002002F085FF2EE019
:1009A000E4B2012C04D14FF4005002F07DFF26E0A8
:1009B000E4B2022C04D14FF4804002F075FF1EE037
:1009C000E4B2032C04D14FF4C04002F06DFF16E0F6
:1009D000E4B2042C04D14FF4004002F065FF0EE0B5
:1009E000E4B2052C04D14FF4204002F05DFF06E094
:1009F000E4B2062C03D14FF4404002F055FFDFF87B
:100A0000500C0470E4B2DFF84C0C50F824004FF4A2
:100A10007A71B0FBF1F08008DFF8741D086010BD3A
:100A200010B5DFF8341C096851F48071DFF8282C08
:100A30001160DFF8241C09688905FAD5DFF8D01C9D
:100A4000DFF8CC2C12680A60DFF8C41C0C68C0B256
:100A5000FFF79DFF10BD00B58DB002200290002071
:100A60008DF80E0001208DF80D0000208DF80F008C
:100A700002208DF80C0002A9DFF8E80302F0ACFFB9
:100A80000820009000208DF8060001208DF8050058
:100A900000208DF8070002208DF8040000A9F1481D
:100AA00002F09AFF01220121EE4802F0F2FF01223A
:100AB0000321EC4802F0EDFF0121012002F04DFF7F
:100AC0000020ADF828000020ADF830000020ADF87F
:100AD0002A004FF400700B900AA95FF0804003F0E9
:100AE000F1FA7020ADF81C000120ADF81E00DFF80F
:100AF000F00C008808900020ADF8240007A95FF0F2
:100B0000804003F04EFB6020ADF810000120ADF8EE
:100B10001200002005900020ADF8180004A95FF035
:100B2000804003F01DFB08215FF0804003F05AFB7A
:100B300008215FF0804003F05FFB01215FF08040FF
:100B400003F0F2FADFF8E40D008850F00100DFF85E
:100B5000DC1D08801C20FFF7CDFA01215FF08040EA
:100B600003F0F0FA0DB000BD80B50421BD4802F0DD
:100B700085FF00280DD0DFF86C0CDFF86C1C0978BD
:100B80000160DFF8680C0088401CDFF8601C0880FA
:100B900003E0DFF8500C00210160DFF8140E00883C
:100BA0004FF6FE710840DFF8081E088001BDDFF82F
:100BB000380C0078052803DADFF82C0C05210170C9
:100BC000DFF82C0C0088B52807DBDFF81C0C007858
:100BD000401CDFF8141C087010E0DFF8140C0088CB
:100BE00050280BDADFF8000C0078062806DBDFF867
:100BF000F80B0078401EDFF8F01B0870DFF8E80BF8
:100C00000078112803DBDFF8E00B1021017070473A
:100C100018ED00E000B58BB04FF48070029000201A
:100C20008DF80E0001208DF80D0000208DF80F00CA
:100C300001208DF80C0002A9254802F0CDFE4FF4EA
:100C40008040009000208DF8060001208DF80500FE
:100C500000208DF8070002208DF8040000A91C4830
:100C600002F0BAFE03220E21194802F012FF012100
:100C7000042002F062FE0020ADF81C000020ADF858
:100C800024000020ADF81E002020089007A9DFF8FE
:100C9000540D03F017FA6020ADF810000120ADF8F4
:100CA0001200002005900020ADF8180004A9DFF81C
:100CB000340D03F055FA0821DFF8280D03F092FAFD
:100CC0000121DFF8200D03F02FFA0BB000BD00006A
:100CD0000004024000080240000C024080B5C0B28F
:100CE000DFF8D01C31F81000DFF8FC1C086001218F
:100CF000DFF8F00C03F026FADFF8DC0D4FF480711A
:100D0000018001BD001002400014024080B5DFF8F0
:100D1000DC0C4FF480710180DFF8CC0C0021016005
:100D20000021DFF8C00C03F00DFADFF8B00D002150
:100D3000017001BD00B583B02020009000208DF827
:100D4000060001208DF8050000208DF80700012025
:100D50008DF8040000A9DFF83C0A02F03DFE07BD53
:100D600000B583B00820009000208DF80600012017
:100D70008DF8050000208DF8070001208DF8040093
:100D800000A9DFF85C0D02F027FE07BD2038024005
:100D90000C00014000B583B04FF4004000900020EB
:100DA0008DF8060001208DF8050000208DF8070061
:100DB00001208DF8040000A9DFF8D80902F00CFE2C
:100DC00007BD00000C04014000B583B04FF4007073
:100DD000009000208DF8060001208DF8050000200D
:100DE0008DF8070001208DF8040000A9DFF8A409A0
:100DF00002F0F2FD07BD00001404014000B583B00D
:100E00004FF40050009000208DF8060001208DF86E
:100E1000050000208DF8070001208DF8040000A9CE
:100E2000DFF8BC0C02F0D8FD07BD00B583B04FF46D
:100E30008050009000208DF8060001208DF80500FC
:100E400000208DF8070001208DF8040000A9DFF8CC
:100E5000900C02F0C1FD07BD00E100E080E100E080
:100E600000E400E0000002400004014020040020F3
:100E70001C030020DFF86C2C4FF400431380C9B230
:100E8000002905D1DFF85C1C4FF400720A8004E0F1
:100E9000DFF8B41D4FF400720A80C0B210F0800178
:100EA000012905DBDFF8301C4FF400520A8004E012
:100EB000DFF8381B4FF400520A80DFF8301B4FF484
:100EC00080520A80DFF8101C4FF480520A80C0B2B2
:100ED00010F04001012905DBDFF8FC1B4FF4005244
:100EE0000A8004E0DFF8041B4FF400520A80DFF8A8
:100EF000FC1A4FF480520A80DFF8DC1B4FF480525A
:100F00000A80C0B210F02001012905DBDFF8C81B00
:100F10004FF400520A8004E0DFF8D01A4FF4005278
:100F20000A80DFF8C81A4FF480520A80DFF8A81B45
:100F30004FF480520A80C0B210F01001012905DB85
:100F4000DFF8941B4FF400520A8004E0DFF89C1A8B
:100F50004FF400520A80DFF8941A4FF480520A804E
:100F6000DFF8741B4FF480520A80C0B210F0080101
:100F7000012905DBDFF8601B4FF400520A8004E012
:100F8000DFF8681A4FF400520A80DFF8601A4FF455
:100F900080520A80DFF8401B4FF480520A80C0B2B2
:100FA00010F00401012905DBDFF82C1B4FF400527F
:100FB0000A8004E0DFF8341A4FF400520A80DFF8A8
:100FC0002C1A4FF480520A80DFF80C1B4FF4805229
:100FD0000A80C0B210F00201012905DBDFF8F81A1F
:100FE0004FF400520A8004E0DFF8001A4FF4005278
:100FF0000A80DFF8F8194FF480520A80DFF8D81A17
:101000004FF480520A80C0B210F00100012805DBC5
:10101000DFF8C40A4FF40051018004E0DFF8CC0986
:101020004FF400510180DFF8C4094FF48051018072
:10103000DFF8A40A4FF480510180DFF80C0C4FF464
:1010400000410180704700003C04002010B50400FE
:101050000800002150F04000C0B2FFF70BFF002154
:10106000062000FB04F050F08000C0B2FFF702FF42
:1010700010BD38B50024002500210020FFF7E6FF51
:10108000002005000FE00121E4B2EDB25420DFF8AA
:10109000382D00FB0520205CFFF7ECFE641CE4B259
:1010A000542CF0DB6D1CEDB2062D01DA0024F6E7BE
:1010B00031BD0000E80300203B0400200020002197
:1010C000002211000DE0C0B2C9B25422DFF8F83C92
:1010D00002FB013200238354401CC0B25428F2DBCF
:1010E000491CC9B2062901DA0020F6E77047000062
:1010F0002C02002080B5FFF71DFEFFF731FEFFF741
:1011000049FEFFF761FEFFF779FEFFF78EFEDFF87D
:10111000380B20210180DFF8300B4FF400410180B3
:10112000DFF8C80808210180DFF864060068322172
:101130004843FFF756F8DFF8A00908210180FFF7C0
:10114000BDFF00212120FFF795FE0021B920FFF708
:1011500091FE0021B720FFF78DFE00211420FFF73C
:1011600089FE00210620FFF785FE00212020FFF7E1
:1011700081FE00210C20FFF77DFEFFF77AFF01BD05
:101180002000002010040020DFF8580920210180F1
:10119000DFF8580808210180DFF848094FF40041C2
:1011A0000180DFF840094FF400710180DFF83C084E
:1011B0004FF400510180DFF834084FF48051018072
:1011C000DFF81C09006850F0C000DFF8141908604F
:1011D000DFF8C005006850F04040DFF8B81508603F
:1011E000DFF8B005006850F44020DFF8A81508606B
:1011F000DFF8EC08006850F04060DFF8E4180860A1
:10120000DFF8DC08006850F04070DFF8D4180860A0
:10121000704700000004002008040020F0030020B4
:10122000F80300200000594024040020000024405E
:10123000F3B500209DF80410082291FBF2F303FBA4
:101240001213180000219DF80420082392FBF3F2EA
:10125000110000239DF807201300C0B2002800D021
:101260005B1C00225B181A00D2B2072A00DB0622A0
:1012700000239DF805409DF806502C192300DBB291
:10128000552B00DB542300250024002600270C00EA
:1012900000E0641CE4B2D2B2944280F08B809DF8EE
:1012A00005503AE09DF80660E4B2C9B2671A7F1EA5
:1012B000EDB207FB06569DF80570F61B009FF65D24
:1012C000F6B2D0F108073E419DF80670E4B2C9B20B
:1012D000B4EB010CEDB20CFB07579DF805C0B7EB62
:1012E0000C07DDF800C017F80C70FFB287403E43D2
:1012F000EDB2E4B25427DFF8D0CA07FB04C7EDB261
:10130000E4B25FF0540CDFF8C0EA0CFB04EC15F813
:101310000CC056EA0C06EE556D1CEDB2DBB29D42D8
:10132000B7D2C0B2002819D1EDB2E4B25426DFF82A
:10133000987A06FB04769DF80670E4B2C9B2B4EB65
:10134000010CEDB20CFB07579DF805C0B7EB0C077D
:10135000DDF800C017F80C70AF55DDE7E4B2C9B294
:101360008C420FD19DF80660E4B2C9B2671AEDB2A3
:1013700007FB06569DF80570F61B009FF65DF6B25A
:101380008640B5E7E4B2D2B2561EB4428AD19DF887
:101390000660E4B2C9B2671A7F1EEDB207FB0656BB
:1013A0009DF80570F61B009FF65DF6B2D0F10807B8
:1013B0003E419DE7F3BD10B40021002200231A0036
:1013C00012E0C9B2D2B25423DFF8FC4903FB024356
:1013D000D2B25424C9B204FB0214245CCC54491C7C
:1013E000C9B25429EDDB521CD2B2062A01DA00211F
:1013F000F6E710BC704700002E00002080B5DFF833
:10140000CC1900220A70DFF8C41900224A70DFF8F4
:10141000BC1900228A70DFF8B4190022CA70DFF804
:10142000AC1900220A71DFF8A41900224A71DFF812
:101430009C1900228A71DFF894190022CA71DFF822
:101440008C1900220A72DFF8841900224A72020005
:10145000C5A1DFF8780902F0D9FE01BD2C040020F7
:1014600010B5C0B2E02828DB10F12004DFF86009D5
:101470004171DFF85C090271DFF854090B218171B9
:10148000DFF84C090121C171E4B20C20DFF84419E6
:1014900000FB0410DFF838190860DFF83429D2E9BE
:1014A0000001FFF7C5FEE4B20C20DFF8281900FBAD
:1014B0000410C07A401CC0B22BE0C0B2B0F13003BF
:1014C0000A2B20D2B0F13004DFF804094171DFF8B3
:1014D00000090271DFF8F80805218171DFF8F008D2
:1014E0000121C171E4B20520DFF8EC1800FB041003
:1014F000DFF8DC180860DFF8D828D2E90001FFF730
:1015000097FE062005E0C0B2202801D1042000E0AB
:10151000002010BD000008080400080808000808A2
:101520002E0400200C0008081000080830040020D9
:1015300014000808180008082DE9F04104000D0007
:10154000160000275FF000080CE03200D2B218EB62
:101550000501C9B2FFB2385DFFF782FF401C10EBF6
:1015600008087F1CFFB2385D0028EED14046C0B2AB
:10157000BDE8F08170B400230022C9B2082491FBB9
:10158000F4F42300C9B2082491FBF4F505FB14150B
:101590002A00C0B2DBB25421DFF82C4801FB034122
:1015A0000400E4B2DBB25425DFF81C6805FB0363DA
:1015B000E35C012414FA02F21A43425470BC7047EF
:1015C0002DE9F04104000D0016001F00761C7F1C61
:1015D0000DE02900C9B24046C0B2FFF7CBFF18F1B9
:1015E00001085FFA88F8F6B2B045F2D36D1CEDB28F
:1015F000FFB2BD4201D2A046F3E7BDE8F08170B46E
:1016000000230022C9B2082491FBF4F42300C9B2DC
:10161000082491FBF4F505FB14152A00C0B2DBB2D7
:101620005421DFF8A44701FB03410400E4B2DBB21C
:101630005425DFF8946705FB0363E35C012414FA87
:1016400002F25A40425470BC704700003804002037
:101650002F00002000000020003802402DE9F0415A
:1016600004000D0016001F00761C7F1C0DE02900F1
:10167000C9B24046C0B2FFF7C2FF18F101085FFAD5
:1016800088F8F6B2B045F2D36D1CEDB2FFB2BD42A0
:1016900001D2A046F3E7BDE8F081DFF8400700681B
:1016A00050F00100DFF834170860DFF830070068F9
:1016B0008007FAD5DFF82807006850F40070DFF8DB
:1016C00020170860DFF81C07006850F00100DFF801
:1016D00014170860DFF8100700684006FAD5DFF835
:1016E000AC0C006830F04070DFF8A01C0860DFF838
:1016F000F406006830F40060DFF8E8160860DFF8F0
:101700008C0C006850F44030DFF8801C0860704793
:101710000838024080B5DFF8C4160968890707D485
:10172000DFF8B816096851F00101DFF8B026116042
:10173000DFF8A81609688907FAD5DFF8A81609683E
:1017400051F00101DFF89C261160DFF89C16096852
:101750004906FAD5022301220100C9B2DFF8880642
:1017600002F06EFD01BD000025640000DFF8740684
:10177000006840084000DFF86C160860DFF85C067F
:10178000006840084000DFF8541608607047000009
:10179000240000200000024010B400210022002399
:1017A0001A000023190011E0DFF838361B6853F0E7
:1017B0008043DFF830462360DFF82C361B689B0738
:1017C000FAD5DFF8A03D1B689A18491CC0B28142C7
:1017D000EADBC0B2B2FBF0F080B210BC7047000090
:1017E00028000020380000403D0400203204002082
:1017F0003404002038B50C000025C0B2FFF78AFF82
:101800002000C0B2FFF7C8FF0500FFF7AFFF2800B8
:1018100080B232BD38B50C210820FFF7EBFFDFF8AE
:10182000701B08800C210720FFF7E4FF02F064F929
:1018300004000D00DFF8580B008802F05DF902008B
:101840000B002000290002F005FA0022DFF8443BDB
:1018500002F03AFB02F0D2F902F044F9DFF8382B3B
:10186000DFF8383B02F030FB5FF06632DFF8303BE8
:1018700002F050F902F0C2F902F034F90022DFF868
:10188000243B02F0E7F902F0B9F9DFF81C1B0880ED
:10189000DFF8180B007800282DD1DFF80C0B00883A
:1018A000C938952823D2DFF8B40D0078092816DB53
:1018B000DFF8A80D00210170DFF8F40A0078002895
:1018C00019D1DFF8F00A0078022814D1DFF8E00A15
:1018D0000F210170FFF743F8FFF718FA0BE0DFF86C
:1018E0007C0D0078401CDFF8741D087003E0DFF801
:1018F0006C0D0021017031BD00B583B04FF4007054
:10190000009000208DF8060001208DF805000020D1
:101910008DF8070001208DF8040000A9704802F03E
:101920005BF86D484FF40071018007BD0C0000406A
:1019300000B585B00120029003208DF80D00002035
:101940008DF80F0003208DF80C0002A9644802F006
:1019500043F80420009000208DF8060001208DF847
:10196000050000208DF8070001208DF8040000A973
:101970005B4802F031F8DFF8B40D0421018005B0B6
:1019800000BD00B583B04FF40040009000208DF8FA
:10199000060001208DF8050000208DF807000120C9
:1019A0008DF8040000A9DFF8C00B02F015F807BDA0
:1019B000100000404074000800B583B01020009073
:1019C00000208DF8060001208DF8050000208DF81C
:1019D000070001208DF8040000A9DFF8E00D01F0F8
:1019E000FBFF07BD00080140380801401A0402400F
:1019F00080B5DFF8780B006850F00400DFF86C1B4E
:101A00000860DFF86C0B00210160DFF8680B002133
:101A10000180DFF8640B00210180DFF8A40D0021B4
:101A20000180DFF83C0C40F2FF110180DFF8340C3C
:101A300001210160DFF8880D00884FF6EF71084042
:101A4000DFF87C1D0880DFF8780D00884FF6FD7107
:101A50000840DFF86C1D0880DFF8640D00884FF641
:101A6000FF410840DFF8581D0880DFF8540D00885A
:101A70004FF67F710840DFF8481D0880DFF8400D01
:101A800000884FF6F7710840DFF8341D0880DFF852
:101A9000200C008850F00100DFF8141C0880DFF8EB
:101AA000200D008850F00400DFF8141D0880DFF8D6
:101AB000040C00884FF6FE710840DFF8F81B088020
:101AC000DFF8FC0C008850F00100DFF8F41C0880FF
:101AD0001E20FEF70FFB01BD180402403E0400204B
:101AE000000402401A00024080B5DFF8880A00882E
:101AF0004FF6FE710840DFF87C1A0880DFF8300CE2
:101B00000078002836D1DFF82C0C0078002827D187
:101B1000DFF8240C0078012822D1DFF8200C0068BF
:101B2000DFF81C1C0968884215D247481021018043
:101B3000DFF8F80B4FF400410180DFF8000C00687B
:101B4000401CDFF8F81B08600F20FEF74AFBDFF8A7
:101B5000F40B10210180DFF8DC0B012101703DE066
:101B6000DFF8BC0D4FF400410180DFF8C80B002105
:101B7000017033E0DFF8B80B0078022829D1DFF8D4
:101B8000B40B007800281AD12F4810210180DFF80B
:101B90009C0B4FF400410180DFF8A00B0068401C53
:101BA000DFF8981B08600120FEF71BFBDFF8940BA1
:101BB00010210180DFF87C0B012101700EE0DFF8BD
:101BC000600D4FF400410180DFF8680B00210170C7
:101BD00004E0DFF84C0D4FF40041018001BD10B569
:101BE000DFF8E00B0078002828D0DFF8D80B007869
:101BF000DFF8D41B11EB800050F8040C401E01F0FC
:101C00007BFFDFF8284CD4E9002302F03FFA10D222
:101C1000DFF81C0B0078401CDFF8141B0870DFF89D
:101C2000100B007805280DD1DFF8040B012101709D
:101C300008E0DFF8FC0A0021017003E0DFF8F00A99
:101C40000021017010BD00001800024038B5DFF817
:101C50005C07007801282AD1DFF8280C0078401CA6
:101C6000DFF8201C0870DFF81C0C0078082803DB64
:101C7000DFF8100C002101700024DFF8080C007858
:101C8000E4B2844245D2E4B2072000FB04F0D0F174
:101C90002F03DBB25322E4B2072000FB04F0D0F1A3
:101CA0002A01C9B25220FFF78BFC641CE5E7DFF87C
:101CB000F8060088B0F5AF7064214843462190FBD8
:101CC000F1F52DB2E800642190FBF1F52DB2002D65
:101CD00000D500252DB2082D00DB0725002412E0D9
:101CE000E4B2072000FB04F0D0F12F03DBB2532253
:101CF000E4B2072000FB04F0D0F12A01C9B252205F
:101D0000FFF75EFC641C2000C0B200B22DB2A842F6
:101D1000E6DB31BDF8B504000800002500270026E9
:101D2000FFF76CFB002005000920060048E036B2F2
:101D30002648305C30380A2841D236B22348305C1D
:101D4000B0F13007E4B2EDB20B2000FB15402049A2
:101D500048711F48002101711D480B2181711C48E9
:101D60000121C171FFB20B20DFF8B81B00FB071087
:101D700017490860164AD2E90001FFF759FAE4B2A0
:101D8000EDB20B2000FB15401149487110480821A5
:101D900001710F480B2181710D480121C171FFB202
:101DA0000B20DFF8801B00FB071000F26E000849D3
:101DB0000860074AD2E90001FFF73AFA6D1C761E67
:101DC00036B2002EB3D5F1BD34000020DC03002074
:101DD000180400203C670008AC710008003802407D
:101DE0002038024008240140002401402DE9F84336
:101DF0000027002500265FF0000800245FF000099E
:101E0000DFF8AC0BFFF7D7FADFF8A80B0078012852
:101E10003DD0DFF8182AD2E9000101F0EFFE0400FE
:101E2000DFF8940B844201DBDFF8904B42F20F7035
:101E3000844226DA642094FBF0F100FB1149494604
:101E40004120FFF767FFB9F10A0F03DA00213620BE
:101E5000FFF760FF642094FBF0F12720FFF75AFFA3
:101E60000E213320FFF786FB0F213320FFF782FB83
:101E70000E213420FFF77EFB0F213420FFF77AFB81
:101E800005E0642094FBF0F14120FFF743FFDFF809
:101E9000300BD0E9002300205FF0804102F014F8FD
:101EA00004000D00DFF81C0B006801F01BFE22008F
:101EB0002B0002F009F80022DFF80C3B01F0CAFE0B
:101EC00001F09CFE040000252000FFF797FA092688
:101ED00013E0DFF8540A305C00280DD01D22EDB26B
:101EE000072000FB05F0D0F14901C9B2DFF8380A3C
:101EF000305CFFF7B5FA6D1C761E002EE9D5002682
:101F00000AE01D22072000FB06F010F11F01C9B2F4
:101F10003020FFF7A5FA761CEDB2D5F10700864216
:101F2000EFDBDFF8A80A0078002801D0012700E0E5
:101F30000027DFF89C0A046800252000FFF75EFAFE
:101F4000092616E0DFF8E009305C002810D0D7F150
:101F50002902D2B2FFB2D7F14900EDB2072101FB4D
:101F60001501C9B2DFF8C009305CFFF779FA6D1CC2
:101F7000761E002EE6D500260DE0D7F12902D2B25A
:101F8000FFB2D7F13B00072101FB0601C9B23020A7
:101F9000FFF766FA761CEDB2D5F103008642ECDB62
:101FA000DFF8280A007800280CD0DFF8200A007833
:101FB000401EDFF8181A08702F234D2227213920E0
:101FC000FFF74CFB00250024DFF8580B0078461E75
:101FD0000BE0DFF8540B30F81680192098FBF0F86E
:101FE000444500DA44466D1C761EEDB21B2D01DA25
:101FF000002EEED53B260BE0DFF82C0B30F81680D8
:10200000192098FBF0F8444500DA44466D1C761E12
:10201000EDB21B2DF0DB641C0025DFF8080B007807
:10202000461E0DE0D7F12D01C9B2D5F11A00C0B29C
:10203000FFF7A0FA7F1CFFB24745F3DB6D1C761E4D
:10204000EDB21B2D0EDA002E0CD4DFF8DC0A30F8CE
:10205000160090FBF4F8B8F11A0F01DB5FF01908D5
:102060000027E8E73B260DE0D7F12D01C9B2D5F1F5
:102070001A00C0B2FFF77EFA7F1CFFB24745F3DBC0
:102080006D1C761EEDB21B2D0CDADFF89C0A30F8C1
:10209000160090FBF4F8B8F11A0F01DB5FF0190895
:1020A0000027EAE700252000FFF7A8F9092613E03A
:1020B000DFF87408305C00280DD02922EDB207202B
:1020C00000FB05F0D0F12D01C9B2DFF85C08305CEF
:1020D000FFF7C6F96D1C761E002EE9D500260AE032
:1020E0002922072000FB06F010F12601C9B230209A
:1020F000FFF7B6F9761CEDB2D5F102008642EFDBB0
:10210000DFF8B00A0088022190FBF1F4DFF8C00884
:102110000068844242D2132000FB04F0DFF8B018BC
:102120000968491EB0FBF1F0D0F11305EDB26D0066
:102130001421D5F14800C0B2FFF71CFA1521D5F1E2
:102140004800C0B2FFF716FA1621D5F14800C0B218
:10215000FFF710FA1421D5F14900C0B2FFF70AFACF
:102160001521D5F14900C0B2FFF704FA1621D5F1C7
:102170004900C0B2FFF7FEF91421D5F14A00C0B200
:10218000FFF7F8F91521D5F14A00C0B2FFF7F2F9CF
:102190001621D5F14A00C0B2FFF7ECF9FFF756FD62
:1021A000DFF820084068002840F0A380DFF87C2694
:1021B000D2E900010122DFF8003B02F0F7F81BD85A
:1021C000DFF8CC0C00214171DFF8C40C0021017153
:1021D000DFF8BC0C10218171DFF8B40C0221C17151
:1021E000DFF8AC0CDFF84C1B0160DFF8A42CD2E95F
:1021F0000001FFF71DF8C6E0DFF83026D2E9000144
:102200000122DFF8343B02F0D1F81BD8DFF8800C54
:1022100000214171DFF8780C00210171DFF8700CAA
:1022200010218171DFF8680C0221C171DFF8600CA8
:10223000DFF8081B0160DFF8582CD2E90001FEF737
:10224000F7FFA0E0DFF8480C00214171DFF8400CF7
:1022500000210171DFF8380C10218171DFF8300C9A
:102260000221C171DFF8BC0800780F2190FBF1F565
:10227000EDB2042095FBF0F101FB1051002905D1CE
:10228000DFF80C0CDFF8141B01602BE0EDB2681CCA
:10229000042190FBF1F202FB1102002A05D1DFF8C4
:1022A000F00BDFF8FC1A01601CE0EDB2A81C042161
:1022B00090FBF1F202FB1102002A05D1DFF8D00BEE
:1022C000DFF8341B01600DE0EDB2E81C042190FB47
:1022D000F1F202FB1102002A04D1DFF8B40BDFF89F
:1022E0001C1B0160DFF8A82BD2E90001FEF7A0FF5C
:1022F00049E0DFF80C0B046800252000FFF77EF8AA
:10230000092613E0DFF82006305C00280DD00022FB
:10231000EDB2072000FB05F0D0F10701C9B2DFF8EC
:102320000806305CFFF79CF86D1C761E002EE9D580
:10233000002608E00022072000FB06F1C9B2302089
:10234000FFF78EF8761CEDB2D5F102008642F1DB84
:10235000DFF83C0B0F214171DFF8340B00210171D4
:10236000DFF82C0B07218171DFF8240B0121C171EB
:10237000DFF81C0BDFF81C1B0160DFF8142BD2E91F
:102380000001FEF755FFBDE8F18300000424014081
:102390003604002000408F4005C58F3177AD0C40DA
:1023A000669080C0000024402A00002040040020E5
:1023B0003F0400202D0000202DE9F041DFF8D00A75
:1023C0000C214171DFF8C80A08210171DFF8C00A49
:1023D0003C218171DFF8B80A0421C171DFF8B80A25
:1023E0000078002805D1DFF8A80ADFF8B01A0160EC
:1023F00004E0DFF89C0ADFF8A81A0160DFF8902AF1
:10240000D2E90001FEF714FF0025002700265FF047
:1024100000080024DFF8AC030078002827D1DFF89B
:10242000780A0078002806D11B221821DFF8740AE8
:10243000FFF782F888E0DFF8580A20214171DFF8C1
:10244000500A1A210171DFF8480A16218171DFF85C
:10245000400A0121C171DFF8380ADFF84C1A016027
:10246000DFF82C2AD2E90001FEF7E2FE6CE0D54845
:102470000078D54911EB800050F8044CB4F57A7F10
:102480002BDA1B221F21642094FBF0F03030C0B205
:10249000FEF7E6FF64201B22292194FBF0F300FBEA
:1024A00013400A2390FBF3F03030C0B2FEF7D8FFA0
:1024B000642094FBF0F100FB11400A231B22302121
:1024C00090FBF3F403FB14003030C0B2FEF7C8FFFA
:1024D00021212620FFF74EF836E0642094FBF0F42B
:1024E0002000FEF78BFF092707E03FB2DFF8380432
:1024F000385C002800D0761C7F1E3FB2002FF4D538
:10250000F6B2072000FB06F0022190FBF1F8092744
:1025100017E03FB2DFF81004385C002810D01B220F
:102520005FFA88F818F12400EDB2072101FB1501CC
:10253000C9B23FB2DFF8F003385CFEF791FF6D1CC3
:102540007F1E3FB2002FE4D5DFF8FC0C0078002896
:1025500006D0DFF8F40C0078401EDFF8EC1C0870A1
:10256000BDE8F081582401400004024024380240B4
:1025700024080040100800400408004080B5DFF83F
:10258000100904214171DFF8080908210171DFF801
:1025900000094D218171DFF8F8080421C171DFF8CD
:1025A000F8080078002805D1DFF8E408DFF8881A79
:1025B000016004E0DFF8D808DFF8801A0160DFF876
:1025C000D028D2E90001FEF733FEDFF8CC0800780E
:1025D000002810D158480078002806D11B22192164
:1025E000DFF8C008FEF7A8FF2AE01B222021A4A0E4
:1025F000FEF7A2FF24E0DFF8980820214171DFF800
:1026000090081A210171DFF8880816218171DFF81E
:1026100080080121C17148480078002805D1DFF801
:102620007008DFF88418016004E0DFF86408DFF860
:10263000101A0160DFF85828D2E90001FEF7F8FD12
:10264000DFF8080C0078002806D0DFF8000C0078CE
:10265000401EDFF8F81B087001BD00004204002096
:10266000280800402C08004010B5DFF8D809FEF714
:10267000A2FE00240020040011E01923E4B20C2083
:1026800000FB04F010F11902D2B21521E4B20C20C3
:1026900000FB04F01130C0B2FEF792FF641CDFF8BB
:1026A000B00B0078E4B28442E7D3FFF7CFFA10BD55
:1026B0000C0800401408004080B5DFF8980B007843
:1026C000002832D0DFF8D0070078002804D1DFF8E6
:1026D000D00AFEF770FE03E0DFF8C80AFEF76BFED3
:1026E000DFF8B4070078002805D115220621DFF8AD
:1026F000B80AFEF721FFDFF85C0B007801280DD146
:10270000DFF8EC0A007802280FD1DFF8480B00212F
:102710000170DFF8DC0A0121017006E0DFF8340BFC
:102720000078401EDFF82C1B087001BD1804024021
:10273000460400204304002030000020280400202C
:10274000E80300201A00024080B5DFF844070421A6
:102750004171DFF83C0708210171DFF834074B2194
:102760008171DFF82C070421C171DFF82C07007894
:10277000002805D1DFF81807DFF8DC1A016004E053
:10278000DFF80C07DFF8D41A0160DFF80427D2E97C
:102790000001FEF74DFDDFF800070078002805D1A5
:1027A0001B220B21DFF8B80AFEF7C6FEDFF8B40AD9
:1027B0000078401EDFF8AC1A087001BD000002402E
:1027C0000008004045040020E071000880B5DFF8F3
:1027D000840A0078002802D0FFF76EFF09E0DFF8D6
:1027E000700A0078002802D0FFF73EFF01E0FFF7F3
:1027F000FDFADFF8540A0078002801D0FFF7DCFD6D
:10280000DFF8480A0078002801D0FFF7B7FEDFF8AC
:10281000540A0078002801D0FFF796FFFEF729FC44
:10282000DFF8580D0021017001BD0000F003002009
:1028300080B50221DFF8E80A01F020F9002807D16D
:10284000DFF8E00A0078401CDFF8D81A087003E0CF
:10285000DFF8D00A00210170DFF8C80A00783328B9
:102860000DDBDFF8C00A00210170DFF8E00A01216A
:102870000170FEF774F8DFF8080D0021017001BD4A
:10288000E2EAEB004804002080B5DFF8C00A0078D7
:1028900001281AD101F0D7FDDFF8B40A01F09EFD3E
:1028A00048480168DFF8A80A01F0E6FD454841689C
:1028B000DFF8000B01F0E0FDDFF8DC050178DFF860
:1028C000200B01F0D9FD01F0CEFDDFF8800A0021D8
:1028D000017001BDDFF80C0B0078DFF8F01B51F838
:1028E000200041F28931884208DBDFF8F80A0078DD
:1028F000DFF8D81B41F2883241F82020DFF8E40AE3
:102900000078DFF8C81B51F82000002807D5DFF851
:10291000D40A0078DFF8B41B002241F82020704769
:102920001A040240D0700008DC03002080B50221A8
:10293000DFF8EC0901F0A2F8002833D1DFF85C0DD4
:102940000078042826DBDFF8A00A007801280CD1E3
:10295000DFF8900A00781B4951F820001430DFF8A6
:10296000841A0978174A42F82100DFF87C0A0078B7
:1029700004280CD1DFF86C0A0078124951F82000C5
:102980001438DFF8601A09780E4A42F82100FFF780
:10299000A1FF0BE0DFF8040D0078401CDFF8FC1C01
:1029A000087003E0DFF8F40C0021017001BD0000A5
:1029B0006C5B000832000020809698007F9698009B
:1029C000000400201004002040775B414A040020EE
:1029D0002000002038B5FFF7A9FFDFF8BC0400781D
:1029E000002804D1DFF8E80AFEF7E5FC03E0DFF891
:1029F000E40AFEF7E0FCDFF8D40A00680024FEF7E2
:102A0000FDFC092512E0DFF8D00A285C00280CD074
:102A10000E22072000FB04F0D0F13B01C9B2DFF821
:102A2000B80A285CFEF71CFD641C6D1E002DEAD55B
:102A300000250AE00E22072000FB05F010F1260118
:102A4000C9B23020FEF70CFD6D1CD4F104008542A4
:102A5000F0DBDFF8780A40680024FEF7CFFC092598
:102A600012E0DFF8740A285C00280CD01A22072034
:102A700000FB04F0D0F13B01C9B2DFF85C0A285C2E
:102A8000FEF7EEFC641C6D1E002DEAD500250AE061
:102A90001A22072000FB05F010F12601C9B23020F0
:102AA000FEF7DEFC6D1CD4F104008542F0DBDFF89C
:102AB00034090078002806D1162344220C21212055
:102AC000FEF7CCFD05E02223442218212120FEF749
:102AD000C5FDDFF8BC0312214171DFF8B4032721E3
:102AE0000171DFF8AC0330218171E9480121C17126
:102AF000E9480078002804D1E548DFF8881A016029
:102B000003E0E348DFF8801A0160E14AD2E90001FE
:102B1000FEF78EFBFEF7ADFADFF8980C002101708E
:102B200031BD00003B0400202C02002038B5FEF728
:102B3000C5FADFF8580A00880024FEF75FFC092573
:102B400012E0DFF89409285C00280CD0002207204E
:102B500000FB04F0D0F14B01C9B2DFF87C09285C1E
:102B6000FEF77EFC641C6D1E002DEAD5DFF8100A0E
:102B700000780024FEF742FC092512E0DFF858092E
:102B8000285C00280CD00A22072000FB04F0D0F1BA
:102B90004B01C9B2DFF84009285CFEF761FC641CF8
:102BA0006D1E002DEAD5FEF764FADFF8080C00214F
:102BB000017031BD2C04002080B5DFF8FC0B0078DB
:102BC000002875D0DFF8D80A0078002853D1DFF844
:102BD000E80B0078022812D1DFF8080800780028F6
:102BE00004D1DFF800080121017008E0DFF8F407E4
:102BF0000078012803D1DFF8EC0700210170DFF82D
:102C0000B80B007801280ED1DFF8D8070078DFF87C
:102C1000BC1851F82000401CDFF8C8170978DFF80D
:102C2000AC2842F82100DFF8900B007804280ED180
:102C3000DFF8B0070078DFF8941851F82000401E44
:102C4000DFF8A0170978DFF8842842F82100DFF8C0
:102C5000680B007803280ED18F480078002803D134
:102C60008D480121017006E08B480078012802D1CF
:102C7000894800210170DFF8400B007805280DD14C
:102C8000DFF81C0A0078002804D1DFF8140A0121BB
:102C9000017003E0DFF8080A00210170DFF848073F
:102CA000DFF8141B09780170DFF80C0B00210170AC
:102CB000FFF710FE01BD000000388F4080B5DFF83F
:102CC000940500210170DFF89C0500210170DFF8F8
:102CD000780500210170DFF8740500210170DFF82C
:102CE000DC0A40210180DFF8D80A04210180FDF7C9
:102CF00090FDFDF71CFEDFF8CC0A006850F01000D4
:102D0000DFF8C01A0860DFF8C00A006850F002005F
:102D1000DFF8B41A0860FEF7EDF9DFF8B00A0068D2
:102D200050F48060DFF8A41A0860DFF8A40A0221DA
:102D3000017001BDC072000800804840E0720008C8
:102D400080B5FFF7A1FDDFF88C0A04210180FDF7B3
:102D5000DDFFDFF8740A006830F00200DFF8681A5F
:102D60000860DFF8600A006830F01000DFF8541ADD
:102D70000860FDF7F4FDDFF8540A006830F4806065
:102D8000DFF8481A0860FEF7FFF9DFF84C0A002167
:102D90000170DFF8480A4021018001BD607300081E
:102DA0004073000880B5FFF7CBFFDFF8340A0068F6
:102DB00050F48070DFF8281A0860DFF8280A0068ED
:102DC00030F00200DFF81C1A0860DFF8180A00680B
:102DD00050F00100DFF80C1A0860DFF80C0A0068F8
:102DE00050F00400DFF8001A0860DFF8E409002161
:102DF000017020BF01BD00002073000800730008AF
:102E00002404002000B583B00120009000208DF83C
:102E1000040001208DF8050000208DF8070000A9AE
:102E2000DFF8C80900F0D8FDDFF89809DFF8941939
:102E300009680160DFF8B809006850F00100DFF8A8
:102E4000B0190860DFF8AC09006850F00100DFF845
:102E5000A419086001210620FDF764F90620FDF79A
:102E600049F907BDDFF87009007801280FD1E04863
:102E7000007802280BD1DFF880090078002806D0FE
:102E8000DFF874090078401EDFF86C19087070478D
:102E9000180400204874000838040020F06E000870
:102EA000E06F0008307400089873000880B5D048BF
:102EB0000078002868D10121DFF8300900F0DEFD3C
:102EC000012861D1DFF8340900684FF4FA714843F2
:102ED000FDF787F90121DFF8140900F0CFFD012883
:102EE00052D1DFF8180900684FF4FA714843FDF732
:102EF00078F90121DFF8F40800F0C0FD012843D182
:102F0000DFF8F80800684FF4FA714843FDF769F9F3
:102F10000121DFF8D80800F0B1FD012834D1DFF835
:102F2000DC0800684FF4FA714843FDF75AF90121B3
:102F3000DFF8B80800F0A2FD012825D1DFF8BC08B1
:102F400000684FF4FA714843FDF74BF90121DFF8AF
:102F50009C0800F093FD012816D1DFF8A008006856
:102F60004FF4FA714843FDF73CF90121DFF87C0882
:102F700000F084FD012807D1DFF85C080121017011
:102F8000DFF874080A210170DFF86C080078002867
:102F900006D197480078022802D195480121017096
:102FA00093480078002802D1914803210170DFF88E
:102FB0004C0800684FF496714843FDF712F9DFF8AA
:102FC0004008006850F00100DFF834180860DFF8AE
:102FD0003008006801BD00B583B0022000900020D9
:102FE0008DF8040001208DF8050000208DF8070001
:102FF00000A9CB4800F0F0FCDFF8C807006850F0EB
:103000001000DFF8C0170860DFF8BC07006850F058
:103010000200DFF8B4170860DFF8D807006850F046
:103020000200DFF8D017086001210720FDF77AF8C9
:103030000720FDF75FF807BD306A0008646B0008E1
:1030400080730008446500082DE9F843DFF8AC07F9
:10305000006814214843FDF7C4F8002600275FF0FC
:1030600000085FF0000900240025DFF84C07007815
:10307000002840F088800920FEF74CFB002675E010
:103080000820FEF789FB00F037FD04000D00DFF893
:103090007407008800F030FD02000B0020002900BA
:1030A00000F0D8FD0022DFF8603700F00DFF00F0DF
:1030B000A5FD00F017FD04000D00200029000022EE
:1030C000DFF8483700F0E2FF00D202272000290095
:1030D0000122DFF83C3701F069F908D82000290007
:1030E0000022DFF8303700F0D1FF00D205272000A2
:1030F00029000122DFF8203701F058F908D8200014
:1031000029000022DFF8143700F0C0FF00D20127A9
:10311000200029000122DFF8083701F047F908D81C
:10312000200029000022DFF8FC3600F0AFFF00D2BB
:103130000427200029000122DFF8EC3601F036F9DF
:1031400008D8200029000022DFF8E03600F09EFFBA
:1031500000D20327B6B2002E06D0FFB25FFA89F97B
:103160004F4501D05FF00108B946761CB6B2142E67
:1031700086DBFEF7FBFA5FFA88F8B8F1000F02D1A0
:10318000DFF834060770DFF87806006850F00200B8
:10319000DFF86C160860DFF868060068BDE8F183A8
:1031A000546100084C6300081874000880B5284872
:1031B0000078401C2649087025480078042806DB62
:1031C000FDF7A4FDFDF725FBFDF7B1FB0BE0FDF7D7
:1031D000C6FBDFF8AC03002101701D480078401EDB
:1031E000C0B2FDF77BFDDFF8CC050121017001BD08
:1031F0002D000020DFF838060078002804D1DFF821
:1032000030060121017003E0DFF82406002101707F
:103210000E480421017070470B48007800280FD039
:10322000DFF810060078401CDFF808160870DFF899
:10323000040600780E2803DBDFF8F8050021017092
:103240000148062101707047470400204404002013
:103250003E0400203F040020986C0008C46D000864
:103260003874000849040020DFF8CC050068052800
:1032700004D1DFF8C4050A2101604CE0DFF8B8058D
:1032800000680A2804D1DFF8B0051421016042E08B
:10329000DFF8A4050068142804D1DFF89C051E217E
:1032A000016038E0DFF8900500681E2804D1DFF8DF
:1032B00088053C2101602EE0DFF87C0500683C2891
:1032C00004D1DFF874057821016024E0DFF8680597
:1032D0000068782804D1DFF86005F02101601AE069
:1032E000DFF854050068F02805D1DFF84C054FF4ED
:1032F000B47101600FE0DFF840050068B0F5B47FFD
:1033000005D1DFF834054FF43471016003E0DFF8D4
:10331000280505210160DFF82405042101707047AC
:10332000000402404B040020DFF814050068002868
:1033300006D1DFF80C05DFF80C150988016003E001
:10334000DFF8FC0400210160704700004C040020FD
:103350000000080880B50221DFF8EC0400F08EFBC5
:10336000002822D10C210920FEF744FA80B28228DD
:103370001FDADFF8D80400780E280ED1DFF8D00469
:1033800000220023C0E90023DFF8C00400210170FF
:10339000DFF8C004052101700BE0DFF8B00400780D
:1033A000401CDFF8A814087003E0DFF8A004002137
:1033B000017001BD0400080800B583B0042000902E
:1033C00000208DF8040001208DF8050001208DF803
:1033D000070000A9DFF8140400F0FEFA07BD0000A2
:1033E000180008084F0400204E04002080B5DFF8C4
:1033F0006804006850F01000DFF85C140860DFF823
:103400005C0400210160DFF8580400210180DFF82E
:10341000540400210180DFF8500400210180DFF80E
:103420004C0440F2FF710180DFF844041521016073
:10343000DFF8340400884FF6EF710840DFF82814F5
:103440000880DFF8240400884FF6FD710840DFF89B
:1034500018140880DFF8100400884FF6FF41084078
:10346000DFF804140880DFF8000400884FF67F714D
:103470000840DFF8F4130880DFF8EC0300884FF60B
:10348000F7710840DFF8E0130880DFF8E8030088F0
:1034900050F00100DFF8DC130880DFF8CC0300886F
:1034A00050F00400DFF8C0130880DFF8CC03008878
:1034B0004FF6FE710840DFF8C013088001211B2081
:1034C000FCF730FE1B20FCF715FE01BD10040020A8
:1034D000645D00085C5F0008DC03002080B5DFF855
:1034E0009C030078002812D12848DFF8941309883B
:1034F0000180DFF88C0300210180FDF758FBDFF825
:10350000840300210160FDF79BF8FEF768FBFEF7DE
:1035100081F9FFF71FFFFFF78BF9FFF7A3FC1748AF
:1035200001210170D84800883C2814DAD648008868
:10353000C1490968B0EB410F0DD2D4480078401E54
:10354000D2490870D1480078002808D1CF48D04926
:103550000978017003E0CD48CD4909780170C2486F
:1035600000884FF6FE710840BF490880BC480088BB
:103570004FF6FE710840BA49088001BD2C000020BA
:103580003D04002014720008447200083404002036
:1035900000B587B001215FF0805000F0DEF9012016
:1035A00000F0C6FF012000F0B4F9002000F0B1F9EE
:1035B000012000F085F9492000F0DFF90028FAD059
:1035C0005FF4803000F084F97F200590FF200690A2
:1035D0000020049004A800F0B1FF00208DF8030043
:1035E00000208DF8000000208DF8010000208DF8EB
:1035F000020000A9002001F03EF8012000F085F94A
:1036000001F007F85FF4801001F072F95FF48010A8
:10361000029000208DF80C0008208DF80D0001208C
:103620008DF80E0002A801F01FF903208DF80400A8
:1036300000208DF8050000208DF8060001208DF88F
:10364000070001A801F062F9002001F079F84FF4B9
:10365000806001F091F801214FF4804001F0A8F85A
:103660008C48CA2101608B4853210160574800688B
:1036700050F480605549086007B000BD80B57A48B5
:10368000008850F00100784908804FF4804001F034
:10369000BDF85FF4801001F02BF901BD4D0400204E
:1036A0005004002080B57C48FCF79BFD7A48FCF76D
:1036B00098FD7948FCF795FDFCF748FD77480068D0
:1036C00030F48030754908600420FDF7A9F9FDF752
:1036D000A0F8FCF78BFDFFF795FBFDF70BFDFDF761
:1036E000DCFFFFF783FEFFF753FFFCF7E1FDFCF77C
:1036F00095FDFFF761FEFDF7AEF9304840210180EE
:10370000FFF769FCFEF758F9FEF73BF9FEF770F991
:10371000FDF780FAFEF7F0F8FEF70AF90FE0FFF781
:1037200005FAFFF749FA2A480078012801D1FFF786
:1037300039FB27480078032801D1FFF7BFFA584822
:10374000007800282BD11C480078002820D01A4887
:103750000078012801D1FFF74DFD174800780228B5
:1037600001D1FFF781FD14480078032801D1FFF74C
:103770001DFD11480078042801D1FFF74DFD0E48CA
:103780000078052801D1FFF7CFFD0B48002101701B
:10379000084800780128C6D1FFF718F8C3E70548A4
:1037A00000780128BDD13F4800780028B7D1FFF745
:1037B00011F9B6E72C00002039040020180002405F
:1037C00018040240080001400C0401400828004091
:1037D0002D0000201A040240400400201A0002407C
:1037E000047000400070004010ED00E00000024056
:1037F000080401400004014041040020240000208E
:10380000140401403604002000408F400000344082
:103810000000494000C0624000A0744000207C408D
:103820000050844000708740004065400040704078
:103830003000002045040020200000204A04002021
:103840004000004028000020000402403A0400200C
:1038500000040020490400202038024024100140C8
:1038600010100140041001400010014028100140D8
:103870002C1001400C100140141001403E040020A7
:1038800032040020280400202C04002032000020F4
:10389000310000202428004040420F000038024040
:1038A0004C040020500400200021DFF80C21126895
:1038B000110031F460410143DFF8FC000160704702
:1038C000DFF8F81000220A70DFF8F0100870704777
:1038D000002110F44032B2F5403F08D13549096863
:1038E00031F0C04110F0C0421143324A11603449F6
:1038F000096831F44031324A11603149096810F4E5
:10390000403008432E49086070472E49C0B2086015
:1039100070472D49C0B208607047C9B2002905D070
:103920002A49096808432949086005E027490968C8
:1039300031EA0000254908607047C9B2002905D066
:103940002349096808432249086005E020490968BD
:1039500031EA00001E4908607047C9B2002905D04D
:103960001C49096808431B49086005E019490968B2
:1039700031EA000017490860704710B400220023A4
:103980000021C0B24409E4B22200012A02D109494F
:103990000B6801E00A490B68C0B210F01F0233FA4D
:1039A00002F0C00701D5012100E000210800C0B2EB
:1039B00010BC7047003802400438024035380240DD
:1039C00034380240D8064742DC0647421C380240E1
:1039D000203802402438024030B400220023002462
:1039E00000252A0046E0012393400C681C409C42BD
:1039F0003FD1036803241500EDB26D00AC40A34332
:103A0000036003680C791500EDB26D00AC402343F0
:103A100003600B79012B02D00B79022B19D183683B
:103A200003241500EDB26D00AC40A34383608368AE
:103A30004C791500EDB26D00AC4023438360838860
:103A400001249440A343838083888C79944023434A
:103A50008380C36803241500EDB26D00AC40A3431E
:103A6000C360C368CC791500EDB26D00AC40234350
:103A7000C360521C102AB6D330BC70470022008AA3
:103A800089B2084201D0012200E000221000C0B239
:103A90007047F0B400230024D2B211F00705EDB254
:103AA000AD00AA40130089B2CA1010EB820289B29D
:103AB000CD1010EB85052D6A0F2611F00707FFB218
:103AC000BF00BE40B543156289B2CA1010EB820236
:103AD000126A1A43140089B2C91010EB8100046203
:103AE000F0BC7047010040F10980F446404200F00C
:103AF00005F851F000416047010000BF09D0B0FA5D
:103B000080F18840C91CC1F58461090501EBD02111
:103B10004005704770B44FF0004591EA030C44BF74
:103B20006B4000F039BF00BF841A71EB030603D26B
:103B3000001BB141121973414FF4001C1CEB410FE3
:103B400034BF7CEB430443E00C0DA4EB1356352E3D
:103B500050DC45EAC323DB0A45EAC121C912B6F1AC
:103B600020050DDD63FA05F6EB4086EA03051242F7
:103B700018BF45F00105C01851F100010CD213E047
:103B800062FA06F5F2405540F3415A40B340F34023
:103B90005A408018594107D349085FEA30005FEA6C
:103BA000350528BF45F0010501F58011420875F182
:103BB000004250F1000041EB045170BC4FF4001C76
:103BC0001CEB410F38BF70470020090D09057047F5
:103BD0001CEB410F10D252EA43060BD0BCEB410F55
:103BE00005D80C0DAB43661E342EB5DD02E0AB43A9
:103BF0008018594170BC704770BC7047F446400D46
:103C000040EAC120490006D200F014F8004248BF43
:103C10006FF00040604700F00DF84FF0004188421F
:103C20008CBF084640426047400D40EAC120490031
:103C300080F00D8040F00040490DA1F58061491CE5
:103C400005D4D1F11F0154BFC840C01770474FF0D1
:103C500000007047F0B540F2FF7581EA030C0CF0EC
:103C6000004C15EA11541DBF15EA1357AC42AF4280
:103C7000E5E0BC41C1F31301C3F31303801A99417A
:103C800043F4801304D2641E400049418018594116
:103C9000C90241EA5051B1FBF3F603FB1611A2FB36
:103CA0000675D7EBC020A94102D2761E8018594173
:103CB000C90241EA5051B1FBF3FE03FB1E11A2FB06
:103CC0000E75D7EBC020A94103D2AEF1010E8018CA
:103CD0005941890241EA9051760546EA8E2EB1FBA0
:103CE000F3F603FB1611A2FB0675D7EB8020A94162
:103CF00002D2761E80185941C90241EA50514EEA5B
:103D0000060EB1FBF3F603FB1611A2FB0675D7EB0B
:103D1000C020A94102D2761E80185941C90241EA49
:103D20005051B1FBF3F703FB1711A2FB0735D3EB9F
:103D3000C020A94167F100070CBF004247F001070E
:103D400066F3D5274FEA1E31B80814F5806412DDFA
:103D5000BD0775F1004250EB0E5051EB045111F5C7
:103D6000801F5CBF41EA0C01F0BD4CF07F6141F067
:103D7000E0410020F0BDBD076D0840EA0E5041F45F
:103D80008011D4F10104B4F120060ADAC4F120064E
:103D90000200E04001FA06F3E1401843B240154347
:103DA0000EE0342C13DCC6F1200445EA40056D0812
:103DB00020FA06F2154321FA06F0A1400D43002136
:103DC00075F1004250F1000051EB0C01F0BD0020F4
:103DD0005FEA0C01F0BDCFB992185B41B3FA83F7EB
:103DE00004BFB2FA82F6BF190B3FB7F120062FBF0E
:103DF00002FA06F3BB40C7F1200622FA06F638BFE6
:103E00003343BA401CB1E419641E33E77F4231F0FA
:103E10000041B1FA81F404BFB0FA80F6A4190B3C5A
:103E2000B4F120062FBF00FA06F1A140C4F120062C
:103E300020FA06F638BF3143A0403C1B1AE7AC42DB
:103E40001ABF05EA1357AF4212E050EA41061CBF01
:103E500052EA4306BFE750EA4107304661461CBFBD
:103E600041EA0551F0BD52EA430C08BFC143F0BD21
:103E700000204FF4001616EB410F98BF16EB430FCE
:103E800008BF16EB410F24BFC14305E016EB430FFB
:103E90000CBF61464CEA0551F0BD10B450F8041B4C
:103EA00081B102681218001D50F8043BDC0744BFC2
:103EB000A9F10104E31852F8044B43F8044B091F1D
:103EC000F9D1EBE710BC7047B0B581EA030C0CF0F8
:103ED000004C40F2FF7515EA11541DBF15EA135747
:103EE000AC42AF4239E0E41923EA455343F480136E
:103EF000C90241F0004141EA505EC7021100A7FB30
:103F0000020200284FF00000EEFB01204FF00001FC
:103F1000E3FB072118BF42F001024018002149418C
:103F2000E3FB0E01A4F580640F0302D2520040416E
:103F3000494154F101046CDD470872F1004250F12F
:103F4000000051EB0451A1F580115CBF41EA0C0166
:103F5000B0BD4CEA05510020B0BD05EA1357AC4294
:103F600014BFAF4241E050EA410E1CBF52EA430E7B
:103F700002E061460020B0BD24423C441BD15FEA10
:103F8000070EF6D0090302BF01460020AEF1140E61
:103F9000B1FA81F7AEEB070401FA07FE0C37C7F15F
:103FA000200100FA07F7C8404EEA000E23EA455305
:103FB00043F48013A2E733F00043B3FA83F704BF5E
:103FC000B2FA82FE77440B3FE41BB7F1200E2FBFFD
:103FD00002FA0EF3BB40C7F1200E22FA0EFE38BFE4
:103FE00043EA0E03BA40641C82E750EA410E14BF54
:103FF00052EA430E6FF000014FF4001717EB430F26
:104000008ABF194617EB410FB5E74CEA055100206E
:10401000B0BDD4F10104B4F120070FDAC4F12007D8
:10402000520828BF42F0010210FA07F501FA07F71B
:10403000E1BF2A43E0403843E1400FE0352C98DCF3
:10404000C7F1200452EA400220FA07F218BF42F0FA
:10405000010231FA07F0A1400A43002172F1004247
:1040600050F1000051EB0C01B0BD50F8041B61B1E0
:1040700050F8042BD30744BFA9F101039A18002379
:1040800042F8043B091FFAD1EFE770474FF4001CD8
:104090001CEB410F94BF1CEB430F09E041EA030CFA
:1040A00050EA4C0C52EA0C0C03D2994208BF9042E1
:1040B000704714BF8B42824270470268531C0360F2
:1040C00011707047002203881A00B0F1804F08D0A9
:1040D000104B984205D0104B984202D00F4B98429B
:1040E00004D14FF68F731A404B881A430C4B9842F9
:1040F00007D00C4B984204D04FF6FF431A400B896F
:104100001A4302804A68C2620988018501218182BE
:10411000704700000004004000080040000C004010
:104120000010004000140040C9B2002904D00188EA
:1041300051F08001018004E001884FF67F72114048
:1041400001807047C9B2002904D0018851F00101F3
:10415000018004E001884FF6FE7211400180704733
:1041600030B400220023048C4FF6EF752C400484F9
:10417000048C2300048B220048F6FF7422400C8834
:1041800052EA04224FF6DF7423400C8953EA0413E9
:104190004C8853EA0413496881630283038430BC6A
:1041A000704730B400220023048C4EF6FF752C407B
:1041B0000484048C2300848B220048F6FF74224080
:1041C0000C8852EA04224DF6FF7423400C8953EA0E
:1041D00004334C8853EA04334968016482830384BE
:1041E00030BC70470022038B1A004FF2FF731A4055
:1041F00052EA0122028370470022838B1A004FF299
:10420000FF731A4052EA0122828370470CB41CB536
:10421000044604A801900A46009401AB00A907488F
:104220007844183000F06EFC009900220A700028D3
:104230005CBF0098001B16BC5DF80CFB7FFEFFFF07
:10424000F0B400240025C9B21E2911DBC46D072576
:10425000B1F11E0603277E43B540AC43DBB2B1F19A
:104260001E050326754313FA05F52C43C46538E093
:10427000C9B2142911DBC4680725B1F1140603275C
:104280007E43B540AC43DBB2B1F114050326754360
:1042900013FA05F52C43C46023E0C9B20A2911DBE7
:1042A00004690725B1F10A0603277E43B540AC43F4
:1042B000DBB2B1F10A050326754313FA05F52C4369
:1042C00004610EE044690725032606FB01F6B540AC
:1042D000AC43DBB2032505FB01F513FA05F52C43CE
:1042E0004461D2B2072A10DA046C1F23551E05263A
:1042F000754313FA05F5AC43C9B2521E05235A4360
:1043000011FA02F52C4304644EE0D2B20D2A10DA01
:10431000C46B1F23D51F0526754313FA05F5AC435F
:10432000C9B2D21F05235A4311FA02F52C43C463C4
:104330003AE0D2B2132A11DA846B1F23B2F10D05D1
:104340000526754313FA05F5AC43C9B20D3A0523AA
:104350005A4311FA02F52C43846325E0D2B2192A9C
:1043600011DA446B1F23B2F113050526754313FAC6
:1043700005F5AC43C9B2133A05235A4311FA02F5C5
:104380002C43446310E0046B1F23B2F1190505268A
:10439000754313FA05F5AC43C9B2193A05235A43DC
:1043A00011FA02F52C430463F0BC70474FF4001C73
:1043B0001CEB410F94BF1CEB430F09E041EA030CD7
:1043C00050EA4C0C52EA0C0C03D28B4208BF8242DA
:1043D000704714BF994290427047000038B50400FE
:1043E00004254FF4004000F085F80500EDB2042DDF
:1043F00026D1DFF8EC00006850F40070DFF8E01020
:104400000860DFF8DC00006850F00800DFF8D0102A
:104410000860002020604FF4004000F06BF80500B9
:10442000DFF8BC00006830F00800DFF8B410086066
:10443000DFF8AC00006830F40070DFF8A41008600A
:104440002800C0B232BDDFF898000068C00709D567
:10445000DFF89000DFF890100160DFF88800DFF8E7
:104460008C1001607047DFF87800006850F00100A0
:10447000DFF86C100860704770B504000D0004266A
:104480004FF4004000F036F80600F6B2042E0DD1CD
:10449000DFF84C00006830F48070DFF844100860EA
:1044A00025604FF4004000F025F806003000C0B24F
:1044B00070BD04200E490968C90701D501200DE02F
:1044C0000B480068C00501D5022007E008480068D5
:1044D00010F4F05F01D0032000E00420C0B2704768
:1044E000043C02400C3C0240EFCDAB8905040302C2
:1044F000183C024010B582B0040004208DF8000082
:10450000FFF7D7FF8DF8000004E0FFF7D2FF8DF82A
:104510000000641E9DF80000012801D1002CF4D198
:10452000002C02D105208DF800009DF8000016BD7A
:104530000149C0B20860704720000E4238B504003F
:104540000025DFF86402CA210160DFF85C02532114
:10455000016000F02BF8002801D100251FE0DFF8F2
:104560003C02006830F04000DFF830120860DFF8ED
:104570002C02006821680843DFF820120860A06858
:10458000DFF820120860DFF81C020068616850EA5A
:104590000140DFF81012086000F032F80125DFF862
:1045A0000802FF2101602800C0B232BD81B00020A6
:1045B000009000200021DFF8F421126852061BD47D
:1045C000DFF8E8015FF0FF310160DFF8E00100682B
:1045D00010F040010098401C00900098B0F5005F7A
:1045E00001D00029F1D0DFF8C4010068400601D5F0
:1045F000012002E0002000E00120C0B201B07047BD
:10460000DFF82802006830F08000DFF82012086030
:10461000704781B00020009000200021DFF8882141
:10462000CA231360DFF8802153231360DFF87C2155
:10463000126832F0A002DFF874311A60DFF86C0102
:10464000006810F020010098401C00900098B0F520
:10465000004F01D00029F1D0DFF85001006880063A
:1046600001D5012000E00020DFF83C11FF220A60A4
:10467000C0B201B0704770B505000C0000260020E4
:10468000002D07D1DFF814010068400601D4002096
:10469000E0700BE0DFF804010068400604D52078E4
:1046A00000F0D7F8060001E00020E070002D0AD0ED
:1046B00020786178090251EA0040A1780843E17846
:1046C00050EA014612E0207800F0B8F80500607862
:1046D00000F0B4F8EDB2C0B2000250EA0545A0788F
:1046E00000F0ACF82843E17850EA0146DFF8180101
:1046F000CA210160DFF8100153210160FFF756FF66
:10470000002801D1002015E0DFF824013040DFF857
:1047100088100860FFF774FFDFF8800000688006EB
:1047200007D4FFF776FF002801D1002002E0012026
:1047300000E00120DFF8D010FF220A60C0B270BD97
:10474000DFF8C410CA220A60DFF8BC1053220A60E6
:10475000DFF848100968C908C900DFF84020116077
:10476000DFF8381009680843DFF830100860DFF818
:104770009800FF2101607047DFF88C10CA220A60A0
:10478000DFF8841053220A60DFF814100860DFF8A5
:104790007800FF2101607047002800400828004091
:1047A0001428004010280040242800400C28004015
:1047B000154ACA231360144A53231360C9B200294F
:1047C0000ED01C49096830F004021143194A1160E7
:1047D0001949096810F004000843174908600EE001
:1047E0001449096830F004029143124A11601249D9
:1047F000096810F0040031EA00000F49086002481F
:10480000FF210160704700002428004000210009BA
:10481000010088B250F080000449096811F080015D
:1048200071EA000001490860704700000C28004050
:104830007F7F7F000828004040280040002101E0E1
:10484000491C0A38C0B20A28FADA50EA0110C0B28C
:1048500070470021C0B202090A235A43110010F028
:104860000F004018C0B270470021234A110082791E
:10487000002A35D0204A126803689A431E4B1A60FA
:104880001E4A126803689A431C4B1A600279511839
:104890000A6803681A430A60194909680268914363
:1048A000174A11601749096802689143154A116057
:1048B000417910290CD11249096802681143104A44
:1048C000116010490968006808430E4908600EE04D
:1048D0000949427951180A6800681043086006E0E7
:1048E000027951180A68006832EA000008607047CF
:1048F00005490860704700000004014004040140BD
:10490000080401400C0401401404014010B40021CB
:1049100000220F23C478002C1FD01649096811F417
:10492000E061D1F5E061090AD1F10402DBB20B418B
:104930004178914082781A401143090102780E4B68
:10494000D154017849110D4A0123007810F01F005D
:1049500013FA00F042F821000AE001784911084AF0
:104960000123007810F01F0013FA00F042F8210034
:1049700010BC70470CED00E000E400E000E100E056
:1049800080E100E070B44FF0004591EA030F44BFAE
:104990006B40FFF7C9B800BF841A71EB030604D25D
:1049A0006E40001BB141121973414FF4001C1CEB07
:1049B000410F34BF7CEB430684E00C0DA4EB13568F
:1049C000362E7DDC012E43DC45EAC32343EA5253F5
:1049D00012BFD20292025B08240545EAC12141EAD6
:1049E0005051D2EBC020994125D407D1B0FA80F6BE
:1049F00010FA06F164D00020203608E0B1FA81F602
:104A0000B140C6F1200220FA02F21143B0404FEA51
:104A1000F474B4EB465434F001064FEA74040AD837
:104A2000D6F50016760D04F00044F04061FA06F267
:104A30005040F1404840C00A40EA415021F0004156
:104A400028BF5FEA500550F1000044EBD12137E068
:104A500045EAC323DB0A45EAC121C90AB6F12005AC
:104A60000EDD42EA0242120CC5F1200603FA06F6F8
:104A7000EB4042EA06056D42984161F100010DE00C
:104A800062FA06F5F240554063FA06FC82EA0C022F
:104A9000F3405A406D42904161EB030111F4801FD5
:104AA00005D1641E620502D06D004041494121F4E8
:104AB0008011430875F1004350F1000041EB0451AF
:104AC00070BC70471CEB410F15D223F0004352EA33
:104AD00043060BD04FEA4C0CBCEB410F04D80C0D35
:104AE000661E342EB7DDEBE7801A994150EA410685
:104AF00008BF0021E4E708BF1CEB430F28BF6FF09D
:104B00000001DDE72DE9F04FA1B0824602AE0020A2
:104B100017461D46029170620DF144080AE017F82D
:104B2000011B0298D0470290002800F08B82706A27
:104B3000401C7062387808B9706A85E22528EED189
:104B40000020F06030617061B061F061306201E0BE
:104B500040F0010017F8011F2029F9D023290DD0BA
:104B60002B2904D02D2906D030290AD00CE040F0A2
:104B7000020080B2EEE740F00400FAE740F00800DF
:104B8000F7E740F01000F4E72A290DD129680A1D43
:104B90002A600968F162002904D5494240F0040006
:104BA000F16280B27F1C13E00021F1620BE0F16A38
:104BB0006FF00043994205D001EB810302EB430102
:104BC0003039F1627F1C3A78A2F130010A29EED324
:104BD00039782E2903D04FF0FF31B1621EE017F86B
:104BE000011F2A2906D129680A1D2A607F1C09682D
:104BF000B16213E00021B1620BE0B16A6FF00043D3
:104C0000994205D001EB810302EB43013039B162D7
:104C10007F1C3A78A2F130010A29EED330860FF6D4
:104C2000C030397800F0EAFD08B117F8010B8DF8B3
:104C30003A009DF83A00682802BF39786829622056
:104C400005D06C2804BF38786C2803D171208DF80A
:104C50003A007F1C11A8B0603978B1F1250023D04B
:104C60001C3871D0001F02286ED9133800F09780CD
:104C7000093869D0801E00F02B81401E00F0D480DE
:104C8000401E022860D9001F00F0CE80401F30D0A7
:104C9000401E00F08480401E20D0C01E09D0801E1F
:104CA0007DD0C01E7BD01BE1F068411CF160252146
:104CB00020E12868011D29600068B26A7060002A3E
:104CC00002D500F0A7FD07E0002100F0BFFD00289D
:104CD0001ABF7168401AB06A30610DE12868011D81
:104CE000296000210068CDE9000111A870607821D9
:104CF000EAE09DF83A00622818D0682806D06A28B1
:104D00000BD06C2819D0712807D016E02868011D37
:104D100029600068716A0180EEE02A68101D286031
:104D20001268706AC117C2E90001E5E02868011D38
:104D300029600068716A0170DEE02868011D296041
:104D40000068716A0160D7E02868C01D20F0070084
:104D5000286000F108022A60D0E90023CDE9002391
:104D6000002B04D5F068421CF2602D220DE0308E3D
:104D7000820704D5F068421CF2602B2205E0C007D0
:104D800005D5F068421CF260202200F80820F06887
:104D900011AA8018706000A800F0E2F9ACE09DF85C
:104DA0003A006C2808BF2A6811D0712808BF2A6809
:104DB00002D02A686A280AD1D21D22F007022A608E
:104DC000144604F108022A60D4E9002303E0131D0D
:104DD0002B6000231268CDE90023682808BF92B237
:104DE00007D0622808BFD2B203D0742818BF7A282F
:104DF00002D10023CDE9002396F8300000075FD5EB
:104E0000DDE90023002B08BF002A59D041F0200023
:104E1000782855D1F068302200F80820401C421C48
:104E2000F26000F808104BE09DF83A0062280CD0C0
:104E3000682810D06A281AD06C2823D0712816D080
:104E400074281FD07A280CD01CE02868021D2A6024
:104E500090F900201AE02868021D2A60B0F90020AD
:104E600014E02868021D2A60002302680FE0286809
:104E7000C01D20F00700286000F108022A60D0E978
:104E8000002304E02868021D2A600268D317CDE9D8
:104E90000023002B04DAF068421CF2602D220DE0A2
:104EA000308E820704D5F068421CF2602B2205E0A8
:104EB000C00705D5F068421CF260202200F80820E7
:104EC000F06811AA8018706000A800F0C0F813E024
:104ED000F068411CF16029680A1D2A60096809E030
:104EE000F068421CF260252200F8082021B1F06829
:104EF000421CF26000F80810F06AF168401AB169CB
:104F0000401A3169401AF169401A7169401A316AD0
:104F1000A0EB010996F830007F1C400710D4202038
:104F20008DF84000002409E0012310AA00A9504692
:104F300000F03EFC002840F08580641C4C45F3DB0B
:104F4000F4680DF1440B0AE01BF8011B0298D047EE
:104F50000290002876D0706A401C7062641E002C9B
:104F6000F2D130208DF840004FF0000BB46909E019
:104F7000012310AA00A9504600F01AFC002861D1B4
:104F80000BF1010BA345F3DB3469D6F804B00AE05A
:104F90001BF8011B0298D0470290002852D0706A7B
:104FA000401C7062641E002CF2D130208DF840004D
:104FB0004FF0000BF46909E0012310AA00A9504644
:104FC00000F0F6FB00283DD10BF1010BA345F3DB0C
:104FD00030697168746900EB010B09E01BF8011B73
:104FE0000298D047029068B3706A401C7062641ED9
:104FF000002CF3D130208DF840004FF0000B346AC4
:1050000008E0012310AA00A9504600F0D1FBC8B95E
:105010000BF1010BA345F4DB96F8300040077FF558
:1050200089AD20208DF84000002400E0641C4C4530
:10503000BFF680AD012310AA00A9504600F0B8FBCE
:105040000028F3D04FF0FF3021B0BDE8F08F2DE9FC
:10505000FA47064682B035690A466F2A08BF082714
:1050600005D041F02000782814BF0A271027D6E980
:1050700000013C2480468946642A18BF692A05D16C
:10508000002903DAD8F1000869EB4909B9F1000FEA
:1050900008BFB8F1000F0CD1306B50B9082F3BD1CD
:1050A00096F83800000737D530203B2485F83B00C0
:1050B00032E0CDE90089FB17404649463A4600F008
:1050C000F1FBB846A8FB0023DDE90089A8EB02024A
:1050D0003032A4F1010AD2B254463A2A03DB9DF8D9
:1050E0000830513B9A180AF8052080465FEA01090A
:1050F00008BFB8F1000F03D0F06861198842D8D317
:10510000082F09D196F83800000705D5605D3028D2
:1051100002D0641E30206055C4F13C00B0616119BA
:10512000F160316B884207DA081A30624FF6EF718E
:10513000308F0840308710E000290ED596F83810DF
:1051400001F01401102908D1716B7269891A326A51
:10515000891A081A0128A8BF306204B0BDE8F08798
:105160002DE9F24F04468EB0D4E90001CDE90201E9
:1051700004AE9DF8380040F02000009061280AD06D
:10518000206B002848BF062004D404BF009867287D
:1051900001D1012020636168C1F30A5040F2FF721F
:1051A00090421CD1080304BF2068002809D10320C5
:1051B000A0619DF8380061381A2836D30FF23461A7
:1051C00008E00320A0619DF8380061381A2829D32F
:1051D0000FF21861E068032200F0DCFBB5E1012862
:1051E00016DA204600F011FC012811DB0027002010
:1051F0000099612920D1E168302201F8012B4A1C75
:10520000E2609DF83820612A0CBF782258220FE016
:10521000626840F2FE3161F31E52471A62604FF03D
:10522000FF30E5E70FF2C051D4E70FF2C451D1E7E8
:105230000A706169891C616110B9002500277BE152
:105240000098612840F09680206B00284CBF2125F3
:10525000451CDDE902012DB26E1CD4E90089002253
:105260000023FEF713FF3ABF89F00040CDE902802A
:10527000CDE902893F1F8DF810200DF1110801E0E2
:1052800000F20708012E32DBDDE9020100220023D3
:10529000FFF78CF82BD21C2102A800F0D7FBDDE928
:1052A0000201FEF7ABFCF61F8146012E09DBFEF77B
:1052B00019FC02460B46DDE90201FFF763FBCDE96D
:1052C000020108F20700072105E009F00F0200F8CB
:1052D000012D4FEA2919B9F1010F01DB491EF4D55F
:1052E000491E5CBF002200F8012DF9D5C8E70DF179
:1052F0001100A8EB00010DF11106A942B8BF0D463F
:105300002DB228002FD4884206DA04A94118497822
:105310000829A8BF0F2100DA002104AA821800E0A2
:105320006D1E12F80139401E8B42F9D00F2904D1AD
:1053300004A941184A78521C4A70002802D504AECC
:105340006D1C3F1D2DB2681E0DD481190A783032B4
:10535000D2B23A2A03DB9DF838303A3B9A1801F86A
:105360000129401EF2D5206B002840F1E580681E1F
:105370002063E1E0DDE9020100220023FEF786FE62
:105380003CBF81F00041CDE902013FB247F29750A6
:1053900078434849DFF820B190FBF1F73FB2C7F1FD
:1053A00007069246012E19DBDDE90289F00707D5D1
:1053B00052465B4640464946FEF786FD8046894692
:1053C00076105046594652465B46FEF77DFD8246B2
:1053D0008B46002EEAD1CDE9028921E07642904643
:1053E000DFF8D89012E0F00707D552465B464046FA
:1053F0004946FEF769FD8046894676105046594673
:1054000052465B46FEF760FD82468B46002EEAD18F
:10541000DDE9020142464B46FEF71CFCCDE90201E4
:10542000009866280CBF07F10A000620216B45187A
:10543000142DA8BF132530208DF810000DF1110692
:10544000DFF87C90012D3DDBDDE90201FEF7ECFB8E
:1054500006F1080104220A23B0FBF3F303EB8306F1
:10546000A0EB4600303001F8010D0A20B3FBF0F04C
:1054700000EB8006A3EB4603303301F8013D521EDA
:10548000E9D1083D01F10806012DDBDBDDE9020170
:10549000FEF7CAFBFEF730FB02460B46DDE90201D0
:1054A000FFF770FA00224B46FEF70EFDCDE9020130
:1054B000CAE700BFA0860100000024400000F03FC2
:1054C00084D797410DF11100301A0DF1110602E059
:1054D000401E7F1E761C31783029F9D0009966294C
:1054E00002D13FB2791C03E065290CBF01210021E4
:1054F000226B8D182DB2A842B8BF05462DB22900E7
:105500001AD4814204DA885D3528A8BF392000DA30
:1055100030208A19521E00E06D1E12F80139491E12
:105520008342F9D0392802D1885D401C8855002972
:1055300002D5761E6D1C7F1C3FB29DF83810009777
:105540002BB23246204600F003F80FB0BDE8F08FD2
:105550002DE9F043054685B01E46D5F830808946D2
:105560001746012E02DA01260FF28C2749F020009F
:10557000BDF93040662808BF641C17D0672840F08A
:10558000818014F1040FC0F28380444580F2808052
:1055900095F83800641C000702D44645B8BFB046F1
:1055A00024B2B8EB040848BF4FF00008E868A969C6
:1055B00024B2012C25DA30234A1C0B54B8F1010F18
:1055C00003DA95F83810090702D52E211154521C20
:1055D000AA6118EB040FB8BFC8F1000424B26142FD
:1055E000A0446962B045B8BF464636B2EE61324665
:1055F000AB693946181800F0CDF9A8EB0600A8628F
:10560000BFE00818A64218DA3246394600F0C2F95F
:10561000A9697118A961A01B6862B8F1010F03DACA
:1056200095F83800000705D5E8682E220A54E86985
:10563000401CE861C5F82880A3E02246394600F006
:10564000A9F9A8692018361BB8F1010F03DA95F8FB
:105650003810090703D5E9682E224254401C36B29F
:10566000A861B045B8BF4646EB6836B23246E1198C
:10567000C01800F08FF9A8693018A861A8EB0600DF
:1056800068627EE04846612816D14FF0700917E045
:10569000464504DA95F83810090758BFB046B8F106
:1056A000010848BF4FF00008B9F1670F14BF4FF071
:1056B00045094FF0650903E0412808BF4FF0500944
:1056C000A969E86817F8013B0B544A1CB8F1010FAF
:1056D00005DA95F83810090758BFAA6117D52E21A9
:1056E0001154531CAB61B8F1010F10DB761E36B2BA
:1056F000B045B8BF464636B232463946181800F0B3
:1057000049F9A8693018A861A8EB06006862A86981
:10571000E9684718200007F8019B03D42B2007F8FD
:10572000010B03E02D2107F8011B444200260DF177
:10573000080808E00A2200A800F00EFA019808F80C
:10574000010B761C009C21B20129F3DA022E06DA45
:1057500049F02000652804BF302007F8010B4EB93E
:10576000302007F8010B07E0761E02A8305C3030CD
:1057700007F8010B012EF7DAA869E9684018381A12
:10578000E86195F8380000F0140010280DD1686920
:10579000A9690818696A0818E9690818A96A08183F
:1057A000696B8842BCBF081A286205B0BDE8F08367
:1057B000F8B504460D4616461F46002004E0E86A88
:1057C000401CE8627F1E002047B116F8011BA86844
:1057D000A047A8600028F2D14FF0FF30F2BD0000D2
:1057E000686A6C747A4C00006E616E004E414E0027
:1057F000696E6600494E4600300000000278C9B26A
:105800008A421AB11CBF10F8012FF9E718BF002017
:105810007047000000F10103810704D010F8011B5C
:1058200089B18107FAD10268B2F10131914311F0D7
:10583000803F04BF50F8042FF6E710F8011B11B1A8
:1058400010F8011BFBE7C01A70470000C9B28307BC
:1058500006D0521E22D310F8013B9942F7D11FE027
:10586000083A13D302F1040241EA012141EA01415D
:1058700050F8043B121F21BF4B40A3F1013C2CEA1E
:10588000030C1CF0803FF3D0C9B2001F083210F89F
:10589000013B521E28BF91EA030FF8D818BF012020
:1058A000401E70471B4213D1094236D12AB18446AB
:1058B000B0FBF2F002FB10C2704700F055B9FCD308
:1058C0000022002370470B000200002100207047D7
:1058D000904271EB030CF6D370B5B1FA81F4B3FAD0
:1058E00083F52C1BA340C4F1200532FA05F633439F
:1058F000A2405FF00046E64002E05B085FEA320249
:10590000841A71EB030524BF204629467641F4D35F
:1059100002000B003000002170BD012ACFD970B504
:10592000140C20D0B1FA81F4B2FA82F5C4F120044B
:105930006419B4F12006D6D3B2405FF00044F440BD
:10594000002502E052085FEA3303C61A71EB020E2B
:1059500024BF3046714664416D41F3D302000B0011
:105960002000290070BD0C46B1FBF2F102FB11458D
:105970002D0445EA1045B5FBF2F402FB145580B244
:1059800040EA0545B5FBF2F002FB105240EA044044
:1059900070BD000062B38B0708D0521E11F8013BA6
:1059A00000F8013B00F024808B07F6D1830740F01C
:1059B000208000BF103A07D330B4B1E83810103A55
:1059C000A0E83810F9D230BC530724BFB1E8081062
:1059D000A0E8081044BF51F8043B40F8043BD2074C
:1059E00024BF31F8022B20F8022B44BF0B78037040
:1059F0007047083A07D3B1E80810083A40F8043B6A
:105A000040F804CBF7D25307E4E730B4436803F01F
:105A1000004201211B031B0B436004BF0368002BE2
:105A200008D10DE00368DD0F45EA440444605B00E3
:105A30000360491E4468E302F4D523031B0B436053
:105A400043681A434260084630BC704770B504464C
:105A50000D466068C0F30A5040F2FF71884207D1DA
:105A60006068000304BF2068002817D0022070BDC2
:105A700020B92046FFF7C9FF012867DA012D0FDBA7
:105A800040F2FF71091A8D420AD36068002847BFAF
:105A900000202F4900202F49C4E90001012070BDDA
:105AA0004142A942616806DA6FF31E51401941EA8A
:105AB0000050606041E0401E63680122451962F3B6
:105AC0001F5305F1350001F000416360352803D311
:105AD00061600020206070BD002215F11F0F04DA04
:105AE00022682360002020356060684213D0521E77
:105AF00025689241C0F12003D2439D4045EAD2720D
:105B000025686668C54006FA03F32B432360636883
:105B100023FA00F06060606808436060B2F1004FF3
:105B200003D80DD12078C0070AD52068401C20601A
:105B3000206828B96068401C60604FF0FF3070BD7D
:105B40006068884204BF20680028F6D1002070BD3C
:105B50000000F0FF0000F07F91FBF2F303FB121155
:105B6000C0E90031704700007047000000000000ED
:105B70000000000000000000000000000000000025
:105B80000000000000000000000000000000000015
:105B90000000000000000000000000000000000005
:105BA00000000000000000000000000000000000F5
:105BB00000000000000000000000000000002A9526
:105BC00000000000000000000000000000000000D5
:105BD00000000000000000000000000000000000C5
:105BE00000000000000000000000000000000000B5
:105BF00000000000000000000000000000000000A5
:105C00000000000000000000000000000000000094
:105C10000000954A10001000100010001000100045
:105C200010001000100010001000100010001000F4
:105C30000000007000502050205020502050205074
:105C400020502050205020502050205020502050D4
:105C500020502050205020502050205020502050C4
:105C60000070000000004AA50000000000000000D5
:105C70000000000000000000000000000000000024
:105C80000000000000000000000000000000000014
:105C90000000000000000000000000000000000004
:105CA00000000000000000000000000000000000F4
:105CB00000000000000000000000A55200000000ED
:105CC00000000000000000000000000000000000D4
:105CD00000000000000000000000000000000000C4
:105CE00000000000000000000000000000000000B4
:105CF00000000000000000000000000000000000A4
:105D0000000000000000000000000000000052A998
:105D10008080808080808080808080808080808083
:105D200080808080808080808080800000000000F3
:105D30002810280000000000000000000000000003
:105D40000000000000000000000000000000000053
:105D50000000000000000000000000000000000043
:105D60000000A9542125253F1E0020302F213F3F50
:105D7000200000000014141414000000003F1F0451
:105D80003E3F0000003F3F0E0C0E3F3F0000003F33
:105D90003F013F3F00000000140E1400000001010D
:105DA0003F3F010100000000303E1F0300000004DF
:105DB0003E3F001E3F213F1E00000000000000008B
:105DC000F8A858A858A8F80808080808080888C8B3
:105DD0000808080808080808F80808080808080853
:105DE0000808080808080808080808080808080833
:105DF00008080808080808080808080808F8A85843
:105E0000A858A8F8000000000000000000000000F2
:105E100000000000FFAA55AA55AAFF80808080805C
:105E20008080909F9080808080808080FF808080B4
:105E30008080808080808080808080808080808062
:105E40008080808080808080808080808080808052
:105E500080FFAA55AA55AAFF00000000000000001C
:105E60000000000000000000FFAA55AA55AAFF008C
:105E70000000000000088444241800000000000016
:105E8000FF00000000000000000000000000000013
:105E90000000000000000000000000000000000002
:105EA0000000000000FFAA55AA55AAFF000000004C
:105EB0000000000000000000000000000F0A0D0AB2
:105EC0000D0A0F080808080808090909090908083F
:105ED000080808080F08080808080808080808083B
:105EE0000808080808080808080808080808080832
:105EF0000808080808080808080F0A0D0A0D0A0F04
:105F00000000000000000000000000000000000091
:105F10000000000000000000000000000000000081
:105F20000000000000000000000000000000000071
:105F30000000000000000000000000000000000061
:105F40000000000000000000000000000000000051
:105F50000000000000000000000000000000000041
:105F6000003F3F252100000000001414141400001D
:105F70000000003F3F0000003F3F060C063F3F008F
:105F800000003F3F090F060000000000140E14003F
:105F9000000001013F3F010100000000303E1F03EF
:105FA000000000043E3F001E3F213F1E0000000095
:105FB0000000000000000000F8A858A858A8F80841
:105FC00008080808080888C8080808080808080811
:105FD000F808080808080808080808080808080851
:105FE0000808080808080808080808080808080831
:105FF0000808080808F8A858A858A8F800000000E1
:10600000000000000000000000000000FFAA55AAE8
:1060100055AAFF80808080808080909F90808080C3
:1060200080808080FF8080808080808080808080F1
:106030008080808080808080808080808080808060
:10604000808080808080808080FFAA55AA55AAFF2A
:106050000000000000000000000000000000000040
:10606000FFAA55AA55AAFF000000000000088444BA
:106070002418000000000000FF00000000000000E5
:106080000000000000000000000000000000000010
:1060900000000000000000000000000000FFAA5502
:1060A000AA55AAFF00000000000000000000000048
:1060B000000000000F0A0D0A0D0A0F080808080862
:1060C0000809090909090808080808080F08080844
:1060D0000808080808080808080808080808080840
:1060E0000808080808080808080808080808080830
:1060F000080F0A0D0A0D0A0F000000000000000042
:10610000000000000000000000000000000000008F
:10611000000000000000000000000000000000007F
:10612000000000000000000000000000000000006F
:10613000000000000000000000000000000000005F
:10614000000000000000000000000000000000004F
:1061500000000000FCFCFCFCFCFCFCFCFCFCFCFC6F
:10616000FCFCFCFCFCFCFC3C3CBCBCBCFCFCFC7C2F
:106170003C7CFCFCFCBCBC3C3CBCBCFCFCFC7C3C5F
:106180007CFCFCFC3C3CBC3C7CFCFC3C3CBCBCFCCF
:10619000FC7C3CBC3C3CFCFCFCFCFCFCFCFCFCFC3F
:1061A000FCFCFCFCFCFCFCFCFF7F7F7F7F7F7F7F97
:1061B0007F7F7F7F7F7F7F7F7F7F7F70707670792B
:1061C0007F7F71787B78717F7F7F7F70707F7F7F2B
:1061D0007F71787B78717F7F70707D7C7E7F7F7030
:1061E0007076777F7F76707970707F7F7F7F7F7F1B
:1061F0007F7F7F7F7F7F7F7F7F7F7FFFFF0000002C
:10620000000000000000000000000000000000008E
:10621000000000000000000000000000000000007E
:10622000000000000000000000000000000000006E
:10623000000000000000000000000000000000005E
:10624000000000000000000000000000000000FF4F
:10625000FF0000000000000000000000000000003F
:10626000000000000000000000000000000000002E
:10627000000000000000000000000000000000001E
:10628000000000000000000000000000000000000E
:1062900000000000000000000000000000000000FE
:1062A000000000FFFFFEFEFEFEFEFEFEFEFEFEFE06
:1062B000FEFEFEFEFEFEFEFEFEFEFEFEFEFEFEFEFE
:1062C0000EEE2EEEEEEEEEEEEEEEEEEEEEEEEEEE8E
:1062D000EEEEEEEEEEEEEEEEEEEEEE0EDE1EFEFE7E
:1062E000FEFEFEFEFEFEFEFEFEFEFEFEFEFEFEFECE
:1062F000FEFEFEFEFEFEFEFF3F3F3F3F3F3F3F3FB5
:106300003F3F3F3F3F3F3F3F3F3F3F3F3F3F3F3F9D
:106310003F3F3F3F303734373737373737373737F7
:106320003737373737373737373737373737373004
:106330003B383F3F3F3F3F3F3F3F3F3F3F3F3F3F78
:106340003F3F3F3F3F3F3F3F3F3F3F3FFCFCFCFC69
:10635000FCFCFCFCFCFCFCFCFCFCFCFC3C3CBC3CFD
:106360007CFCFCFCFC7C3C7CFCFCFCBCBC3C3CBCED
:10637000BCFCFCBCBC3C3CBCBCFCFCFC3C3CBCBC1D
:10638000FCFCFC3C3CBC3C7CFCFCFCBC3C7C7C3C0D
:10639000BCFCFCFCFCFCFCFCFCFCFCFCFCFCFCFC7D
:1063A000FF7F7F7F7F7F7F7F7F7F7F7F7F7F7F7F7D
:1063B00070707670797F7F7F71787B78717F7F7F57
:1063C0007F70707F7F7F7F7F7F70707F7F7F7F7F19
:1063D000707076777F7F7F70707D7872777F7F7F38
:1063E0007E70707E7F7F7F7F7F7F7F7F7F7F7F7FDD
:1063F0007F7F7FFFFF000000000000000000000022
:10640000000000000000000000000000000000008C
:1064100000E0E0000000000000C0E02020E0C0003C
:1064200000000060E000C060C000E060000000000C
:10643000000000000000000000000000000000005C
:1064400000000000000000FFFF000000000000004E
:10645000000000000000000000000000000000003C
:106460000000000000070704040000000003070408
:1064700004070300000000000306030003060300F6
:10648000000000000000000000000000000000000C
:106490000000000000000000000000FFFFFEFEFE04
:1064A000FEFEFEFEFEFEFEFEFEFEFEFEFEFEFEFE0C
:1064B000FEFEFEFEFEFEFEFE0EEE2EEEEEEEEEEE1C
:1064C000EEEEEEEEEEEEEEEEEEEEEEEEEEEEEEEEEC
:1064D000EEEEEE0EDE1EFEFEFEFEFEFEFEFEFEFEFC
:1064E000FEFEFEFEFEFEFEFEFEFEFEFEFEFEFEFFCB
:1064F0003F3F3F3F3F3F3F3F3F3F3F3F3F3F3F3FAC
:106500003F3F3F3F3F3F3F3F3F3F3F3F30373437C5
:10651000373737373737373737373737373737370B
:1065200037373737373737303B383F3F3F3F3F3FCD
:106530003F3F3F3F3F3F3F3F3F3F3F3F3F3F3F3F6B
:106540003F3F3F3F0000000000000000000000004F
:10655000000000000000000000000000000000003B
:10656000000000000000000000000000000000002B
:10657000000000000000000000000000000000001B
:10658000000000000000000000000000000000000B
:106590000000000000002A9500000000000000003C
:1065A00000000000000000000000000000000000EB
:1065B00000000000000000000000000000000000DB
:1065C00000000000000000000000000000000000CB
:1065D000008040C0008080808080000000000000BB
:1065E00000000000000000000000954A00000000CC
:1065F00000000000000000000000FC04F41414146B
:10660000141414141414F404F4141414141414149A
:106610001414F404F4141414141414141414F404BA
:10662000FC00FC02010000FF0088888888880000C8
:1066300000000000000000000000000000004AA56B
:1066400000000000000000000000000000001F101B
:1066500017141414141414141414171017141414F5
:1066600014141414141417101714141414141414E8
:10667000141417101F001F20408000FF0088888816
:1066800088880000000000000000000000000000FA
:106690000000A55200000000000000000000000003
:1066A00000000000000000000000000000000000EA
:1066B00000000000000000000000000000000000DA
:1066C00000000000000000000000000000000101C8
:1066D00000000000000000000000000000000000BA
:1066E00000000000000052A90000000000000000AF
:1066F000000000000000000000000000000000009A
:106700000000000000000000000000000000000089
:106710000000000000000000000000000000000079
:106720000000000000000000000000000000000069
:1067300000000000000000000000A9547E090909C3
:106740007E00000000000005417F494949320000F9
:1067500000000006417F494949360000000000065C
:10676000417F4101030000000000000540417F41DE
:10677000417F414000000008417F495D41630000C6
:1067800000000006417708497F4908774100000969
:10679000224149493600000000000005417F5108B0
:1067A000457F410000000007417F5108457F4100BF
:1067B00000000007417F49085563410000000007C1
:1067C00040413F01417F410000000007417F4508F3
:1067D0001008457F41000009417F4908497F410079
:1067E000000000073E4141413E000000000000055E
:1067F000417F4101417F410000000007417F49097D
:1068000009060000000000063E4141412200000050
:10681000000000050301417F410103000000000763
:106820000147493009070100000000071E21217FB0
:1068300021211E00000000074163550855634100F7
:1068400000000007013F4140417F41000000000778
:10685000010F1110517F410000000007013F41402E
:10686000413F4140413F010B013F4140413F4140D9
:10687000417F410B03417F49484830000000000739
:10688000417F4948483000417F41000A417F4948E3
:106890004830000000000006224149493E00000047
:1068A00000000005417F49083E4141413E0000098A
:1068B000466919497F4100000000000680B5524832
:1068C000006850F480705049086050480068504992
:1068D00008404E4908604C4800684E4908404A4903
:1068E00008604948006830F48020474908604748FC
:1068F000006830F47D004549086047480021016088
:1069000000F005F845485FF00061016001BD82B00C
:1069100000200190002000903B48006850F4803037
:10692000394908603848006810F400300090019838
:10693000401C01900098002803D10198B0F5A06F89
:10694000F0D131480068800302D50120009001E0B9
:10695000002000900098012853D13148006850F081
:1069600004002F4908602E48006850F002002C49AE
:1069700008602B48006850F0010029490860294848
:10698000006850F080502749086027484FF40061A4
:10699000016026480068C006FBD41C481B490968F2
:1069A00001601A48194909680160184817490968BF
:1069B00001601648006830F47D00144908601348EF
:1069C000006850F41100114908600F48006850F049
:1069D00080700D4908600C4800688001FBD50B48A9
:1069E000006880088000094908600848006850F085
:1069F0000300064908600548006810F00C000C28E8
:106A0000F9D102B070470000003802400838024057
:106A10000CC0FF88FEFFFEEE0C38024008ED00E0DF
:106A2000003C0240243802400070004004700040E6
:106A3000FFFFFFFFFF0F0FBF1F0FFFFF0F0FBF0F66
:106A40000FFFFFFFFF0FEF0F0FFFFFFF0F0FBF1F26
:106A50000FFFFF0F0FBF1F4FEFFFFFFF7F1FCF1F66
:106A60007FFFFFFF0F0FFF0F0FFFFFFF0F0FBF1F76
:106A70000FFFFF9F0F6F0F0FFFFFFFFFFFFF1F1F96
:106A80001F1F1C1E1F1C1C1F1F1C1C1F1C1C1F1F2C
:106A90001D1C1D1D1C1C1D1F1F1C1E1F1C1C1F1F21
:106AA0001C1C1F1E1C1D1F1F1D1C1E1E1E1C1D1F0F
:106AB0001F1C1C1D1C1C1D1F1F1C1E1F1C1C1F1F00
:106AC0001D1C1E1C1C1F1F1F1FFFFF0000000000BD
:106AD00000000000000000000000000000000000B6
:106AE00000000000000000000000000000000000A6
:106AF0000000000000000000000000000000000096
:106B00000000000000000000000000000000000085
:106B1000000000000000FFFF808080808080808077
:106B20008080808080808080808080808080808065
:106B30008080808080808080808080808080808055
:106B40008080808080808080808080808080808045
:106B50008080808080808080808080808080808035
:106B6000808080FFFFFFFFFFFFFFFFFFFF0F0FFF92
:106B7000FF0F1FBF0F0FFFFF0F0FEF0F1FFFFF0FC5
:106B80000FFFFF1F0FEFEFEFFFFF7F1FCF1F7FFFF5
:106B9000EFEF0F0FEFEFFFFF0F0FFFFF1F0FEFEFF5
:106BA0000F1FFFFF0F1FBF0F0FFFFFFFFFFFFFFFB5
:106BB000FFFF1F1F1F1F1F1F1F1F1C1C1F1F1C1C31
:106BC0001F1E1C1F1F1C1C1D1C1E1F1F1C1C1F1FEB
:106BD0001E1C1D1D1D1F1F1C1E1E1E1C1F1F1F1CDB
:106BE0001C1F1F1F1F1C1C1F1F1E1C1D1D1C1E1FCA
:106BF0001F1C1C1F1E1C1F1F1F1F1F1F1FFFFF000E
:106C00000000000000000000000000000000000084
:106C10000000000000000000000000000000000074
:106C20000000000000000000000000000000000064
:106C30000000000000000000000000000000000054
:106C400000000000000000000000FFFF8080808046
:106C50008080808080808080808080808080808034
:106C60008080808080808080808080808080808024
:106C70008080808080808080808080808080808014
:106C80008080808080808080808080808080808004
:106C900080808080808080FFFFFFFFFFFFFFFFFF7D
:106CA000FFFFFFFFFFFFFFFFFFFFFFFFFFFFFFFFF4
:106CB000FF0FEF0F0FFFFFFF1F0FEFEF0F1FFFFF84
:106CC000EFAF0F5FFFFF7F1FCF1F7FFFFFFFFFFFB4
:106CD000FFFFFFFFFFFFFFFFFFFFFFFFFFFFFFFFC4
:106CE000FFFFFFFF1F1F1F1F1F1F1F1F1F1F1F1F34
:106CF0001F1F1F1F1F1F1F1F1F1F1D1C1D1D1C1CB3
:106D00001D1F1F1E1C1D1D1C1E1F1F1D1D1C1E1FA9
:106D10001F1C1E1E1E1C1F1F1F1F1F1F1F1F1F1F8C
:106D20001F1F1F1F1F1F1F1F1F1F1F1F1FFFFF00D2
:106D30000000000000000000000000000000000053
:106D40000000000000000000000000000000000043
:106D50000000000000000000000000000000000033
:106D60000000000000000000000000000000000023
:106D70000000000000000000FFFF80808080808015
:106D80008080808080808080808080808080808003
:106D900080808080808080808080808080808080F3
:106DA00080808080808080808080808080808080E3
:106DB00080808080808080808080808080808080D3
:106DC000808080FFFFFFFFFFFFFFFFFFFFFFFFFF50
:106DD000FFFFFFFFFFFFFFFFFFFFFFFF0F0FEF0FA3
:106DE0001FFFFF1F0FEFEF0F1FFFFF9F0F2F6FFF03
:106DF000FF0F0FAFEFFFFFFFFFFFFFFFFFFFFFFFE3
:106E0000FFFFFFFFFFFFFFFFFFFFFFFFFFFFFFFF92
:106E10001F1F1F1F1F1F1F1F1F1F1F1F1F1F1F1F82
:106E20001F1F1F1F1F1F1F1C1C1D1C1E1F1F1E1C82
:106E30001D1D1C1E1F1F1D1D1C1E1F1F1C1C1D1D7C
:106E40001F1F1F1F1F1F1F1F1F1F1F1F1F1F1F1F52
:106E50001F1F1F1F1F1F1F1F1FFFFF00000000001D
:106E60000000000000000000000000000000000022
:106E7000F8F848F8B0000000F8F82808000030786A
:106E8000E8C80000F8F82808000008F8F808000032
:106E900000000000000000000000000000000000F2
:106EA00000000000FFFF80808080808080808080E4
:106EB00080808080808080808080808181808081CF
:106EC00081808081818181808081818180808081B9
:106ED00081818180808081818080808080808080AD
:106EE000808080808080808080808080808080FF23
:106EF000FFFFFFFFFFFFEFEF0F0FEFEFFFFF0F0FA2
:106F00006F0F9FFFFF0F0FAFEFFFFF0F0FAF0F5F71
:106F1000FFFF1F0FEFEF0F1FFFFF0F0FEFEFFFFF41
:106F20007F1FCF1F7FFFFFFFFFFFFFFFFF1F1F1F01
:106F30001F1F1F1F1C1C1F1F1F1F1C1C1F1F1F1F6D
:106F40001F1C1C1D1D1F1F1C1C1D1C1E1F1F1E1C6B
:106F50001D1D1C1E1F1F1C1C1F1F1F1D1C1E1E1E57
:106F60001C1D1F1F1F1F1FFFFF000000000000004F
:106F70000000000000000000000000000000000011
:106F80000000000000000000000000000000000001
:106F900000000000000000000000000000000000F1
:106FA000000000FFFF808080808080808080808063
:106FB00080808080808080808080808080808080D1
:106FC00080808080808080808080808080808080C1
:106FD000808080808080808080808080808080FF32
:106FE000FFFFFFFFFFFFFFFFFFFFFF7F1FCF1F7FA1
:106FF000FFFFFF0F0FFFFFFFFFFF7F1FCF1F7FFF71
:10700000FFFF0F0F6F0F9FFFFFFF0F0F9F3F9F0FA0
:107010000FFFFFFFFFFFFFFFFFFFFFFFFF1F1F1F10
:107020001F1F1F1F1F1F1F1C1E1E1E1C1F1F1F1C7C
:107030001C1D1D1F1F1F1C1E1E1E1C1F1F1F1C1C76
:107040001F1E1C1F1F1F1C1C1F1F1F1C1C1F1F1F60
:107050001F1F1F1F1F1F1FFFFF0000000000000059
:107060000000000000000000000000000000000020
:107070000000000000000000000000000000000010
:107080000000000000000000000000000000000000
:10709000000000FFFF808080808080808080808072
:1070A00080808080808080808080808080808080E0
:1070B00080808080808080808080808080808080D0
:1070C000808080808080808080808080808080FF41
:1070D0000000FC020101010102FC000000000202AC
:1070E000FF000000000000001C1A010101C23C006A
:1070F0000000000C0E818181C23C00000000008075
:10710000601806FF000000000000FF81414141813E
:1071100000000000FC82414141419A1C00000C0328
:10712000010101C13907010000003C62C1818142B7
:107130003C00000000FC020101010102FC00000013
:107140003F4080808080403F000000008080FF80C2
:10715000800000000000C0B088868180C030000040
:1071600000385880808080413E0000080E090808E1
:1071700088FF8808000000385980808080403F00E8
:1071800000003F4080808080403F00000000000001
:10719000FE0100000000001C624180808143661CEB
:1071A000000000385982828282413F003E414141C5
:1071B0003E00427F400042615149462241494936E2
:1071C0001814127F1027454545393C4A494930017A
:1071D00001710D033649494936064949291E000007
:1071E0001E0000003200000064000000C800000023
:1071F000F4010000E8030000D0070000881300003D
:1072000010270000983A0000204E000050C30000F4
:107210009F860100FCFC243C1800009CFCE07C1CC8
:10722000000078FC848484000078FC84848400005E
:10723000FCFC1078EC840000FC7C10F8FC0000FCE6
:107240007C10F8FCFCFC9484000000FCF8107CFC32
:1072500000000078FC8CA4E4E4000000FCFC8080CA
:10726000000000FCFC00000098BCF464000000FC7E
:10727000FC10FCFC10B5074979441831064C7C44DD
:10728000163404E00A68081D511888470146A142D7
:10729000F8D110BD0800000028000000CFCDFFFF8E
:1072A000200400003400002000000000EFCBFFFFAE
:1072B0003400000074020000000000200000000004
:1072C000000000003E4FCFBFCF4F7E000000000007
:1072D0000000CCCC48283312332848CCCC00000026
:1072E00000000000C0300CE2E20C30C000000000E2
:1072F00040B08C83808080B7B7808080838CB04022
:107300000080404080182442241880C0C0800000C3
:1073100001020404023148844831030707030100D5
:1073200000804040801824422418804040800000A3
:1073300001020404023178FC7831020404020100E5
:107340000080C0C080182442241880404080000083
:107350000103070703314884483102040402010095
:107360000080404080183C7E3C18804040800000F7
:10737000010204040231488448310204040201007D
:10738000000000003C7E42427E3C0000007E7C0803
:107390003E7E000000000000003C7E42427E3C0039
:1073A00000007E7E0A020000007E7E0A02000000CD
:1073B0007047FEE7FEE7FEE7FEE77047704770475D
:1073C00080B5F8F7C2FE01BD00F009F8002801D031
:1073D000FFF750FF0020FCF765F900F002F80120EC
:1073E000704700F001B800000746384600F002F888
:1073F000FBE7000080B5C046C046024A11001820D5
:10740000ABBEFBE726000200014880470148004769
:10741000BD68000825740008F0E0E7F0FFE6E5ED40
:10742000E0000000C046C046C046C046FFF7CCFFA3
:10743000E2FBEAEB00000000EEF7E8F9E5EDE00022
:107440000100040007000700022512082452200052
:10745000FFF7AEBFFFF7ADBFFFF7ACBFFFF7ABBFA6
:10746000FFF7AABFFFF7A9BFFFF7A8BFFFF7A7BFA6
:10747000FFF7A6BFFFF7FEBFFFF7FEBFFFF7FEBF98
:10748000FCF7FCB8FFF7FEBFFFF7FEBFFBF70EBD32
:10749000FBF7DABDFFF7FEBFFFF7FEBFF8F742BF0D
:1074A000FFF7FEBFFFF7FEBFFFF7FEBFFFF7FEBF10
:1074B000FFF7FEBFFFF7FEBFFFF7FEBFFFF7FEBF00
:1074C000FFF7FEBFFFF7FEBFFFF7FEBFFFF7FEBFF0
:1074D000F8F7DEBEFFF7FEBFFFF7FEBFFFF7FEBF08
:1074E000FBF7FCBFF9F740BBFFF7FEBFFAF7FCBAAA
:1074F000FFF7FEBFFFF7FEBFFFF7FEBFFFF7FEBFC0
:10750000FFF7FEBFFFF7FEBFFFF7FEBFFFF7FEBFAF
:10751000FFF7FEBFFFF7FEBFFFF7FEBFFFF7FEBF9F
:10752000FFF7FEBFFFF7FEBF0000010000000200F2
:10753000000004000000080000001000000020000F
:10754000000040000024F4001E0000000C020000B7
:0C755000C800A40101023C050104040075
:040000050800742556
:00000001FF
